:020000041100E9
:10300000002373B52B4D2C4C28006361022601F080
:103010005DFA4021FE2221742800284B009601F021
:10302000A7FA002836D1217CFF222800244B0096E5
:1030300001F09EFA00282DD1224BA2899A4226D176
:10304000E389214A93420DD1204B6361204B2268D2
:10305000002A03D1002B01D043CB43C4280001F048
:1030600073FA73BD1B4A934201D00023EFE71A4B5A
:103070001A4A1B68934206D9C02304222800217CE7
:103080009B0001F0EBFA114B6361154BDFE7002366
:103090002374EAE7CC233821AC2228009B01217459
:1030A00001F0DCFA0028F2D10E4B63610E4BE38194
:1030B0000E4BCCE7D443FF1F8063FF1F8C63FF1FC1
:1030C0008E63FF1F5959000083050000F94200116B
:1030D00008BE001182150000A463FF1F87130000C3
:1030E00014BE0011B1430011AAAAFFFFFCBD0011DC
:1030F000F7B5164B0192C318021D002000938823D8
:103100005B05D3181B685C1C1AD09CB2402C18D8E5
:103110008D781E0CAC466746CD782D023D43AE42FD
:1031200006D1019800280ED110000C70240A4C70B2
:1031300003249BB20733A343D218009B9A42DED3E9
:10314000FEBD4432F9E71000FAE7C046FC0F00006C
:10315000802213B503000324019189B25201073183
:103160009B18A14304305A1A88235B05C3181B68B7
:10317000591C03D190429241104016BD99B240298A
:1031800007D80B000733A343C0189042ECD30020AC
:10319000F3E74430F9E7134B134A1B68126810B584
:1031A000FA24934201D81A00F824104BE4021B6859
:1031B0009A4210D813000E4A12689A420ED3013375
:1031C00007D1F823DB029C4203D10A49054808F0E5
:1031D00067FA200010BDFC24E402ECE7FE24E402C0
:1031E000F7E7C04600C0071100D0071100E0071143
:1031F00000F00711FFFFFF7FF0B59BB015000490B2
:103200000391402A00D9A0E006AB59801A80FFF74D
:10321000C2FF0400042816D9002206A9FFF768FFA0
:10322000052810D906AB1B88AB420CD1002D07D066
:10323000514B2A000499C01808F002FD002802D161
:1032400001201BB0F0BD06AB1D8020000699FFF7E2
:103250007FFF041E7BD1069B0793FFF79CFF802313
:103260005B01C618802307001B039E4201D3F8268A
:10327000F60288235B05F31801931B68013302D023
:10328000019808F0BDFA3D49019808F009FA3B1D84
:103290000293331D05938822029B52059B181B68DD
:1032A00008935A1C3CD044219AB20091402A04D879
:1032B0000320D11D814389B2009103991B0C8B42DD
:1032C00024D0402A22D80122300008A9FFF710FF9D
:1032D000021E1BD1380008A9FFF70AFF04000428CA
:1032E00031D9009A059B9B1880225201B218934253
:1032F00040D288235B05C118009A09A808F070FA2B
:103300001D4B009A09A9F01808F0BAFA009A029B1E
:103310009446634402931A4B029AFB189A42BAD31A
:1033200088235B05FC1821680198013908F0B8F979
:10333000200008F065FA039A07AB5A80300007991D
:10334000FFF706FF0400002C03D1002079E70428D2
:10335000FBD988235B05E018069908F0A1F903233F
:10336000EA1C9A4300D16BE7034B0499E01808F07C
:1033700087FA65E70424ECE704000011FFFFFF7FF4
:10338000F80F0000F7B505001400402A21D80027E7
:1033900001AE71803780FFF7FEFE042816D93A008F
:1033A0003100FFF7A5FE042810D93688BC420BD0A7
:1033B000BD4209D0221CB44200D9321C064B92B245
:1033C000C118280008F00CFA30B2FEBDC04300B2AC
:1033D000FBE703204042F8E70400001137B5042260
:1033E00004000D0001A81649FFF7CCFF02000428D5
:1033F0000BD1019BA34208D3AB4204D0104901A8D2
:103400000195FFF7F9FE01203EBD0E4C2368200018
:10341000019308F0F5F9019920000139019108F0B4
:103420003FF980235B01E418074B9C42EED1042254
:10343000034901A80195FFF7DFFE0020E4E7C0463D
:103440005555000000C007110000081130B589B0C3
:1034500008F05EFB10226946254808F031FB254B39
:10346000009A9A420ED1019B029A0F2B33D8002169
:1034700001240698013B08D2002900D00292029B49
:10348000013331D10023029325E0551CF2D1020013
:103490002100EFE710341022200004A908F010FBEF
:1034A000029B013301D1069B0293882304995B059B
:1034B000C918059B06981A03120B049105928142C4
:1034C00003D02B4201D108F08BF9019B013B019302
:1034D000019B002BDED1029B002B03D004930498A8
:1034E0004168084709B030BDE025014C2D03EFE7E6
:1034F0000000011150485936F7B50F4F0F4BFA6DC8
:1035000004001A4084235B001343FB65030010335F
:10351000019300252E00112008F0FAFB0322BB6E58
:103520001340AB4002351E43202DF4D1019B40C413
:10353000A342EED1F7BDC04600F0004000FEFEFF02
:10354000802270B5AD4CAE4BD200002120001C6033
:1035500008F036F92300AB4A88331A60AA4B1A7870
:103560006E23002A00D01133E3620A232365A74BA0
:103570001878A74BA0630138E361C3B2032B01D8CD
:1035800010232362A34B37226361C823DB00A361AE
:1035900023008C331A60082336210F3AE518E163C3
:1035A00023646264E9670439251DE96725003B2629
:1035B000BC352E602500C0352B602500C4352A603F
:1035C00025000636CC352E602500083EC8352E6015
:1035D0002500D03529602100D4310B602100D8317D
:1035E0000A6021000225E0310D6025004221DC3512
:1035F000296025001B3EE4352E602500E8352B6050
:103600002500EC352A6022000525F43215602200E1
:10361000F032116022001831903211602200943291
:10362000136023003C2298331A60AF23DB00236031
:10363000794B2363032805D808F0FAFA33023537AB
:103640001523636096232100FA225B00A360E360E8
:10365000C8332361714BFC319200A3640A6062623B
:103660006F4A704DA2627322E2656D3A6265A2658F
:103670000232E5644A600221616696218900A166F2
:10368000626709210022E166A2676749674A684EBE
:103690002167E2673560032811D808F0C9FA960857
:1036A0009EA61023CDE70E23CBE70C23C9E720000D
:1036B0001A259C30056020000735A03005602000E9
:1036C000A83003602300FA20F8338000186023003C
:1036D0006420A433186023005F38AC3318602300E3
:1036E0000338B03318602300C630B43318602300A9
:1036F0000020B833186023003825FC339D604D4D01
:103700005A665D644C4D9A64DD619625AD001D627C
:103710004A4D9A675D62F53DFF3D9D621E25484A10
:10372000DD6618675867D9651966DA67BE23C02158
:10373000444A5B00E250444B4900635004316250FC
:10374000C4225200A350FA23E4205B000432A350A9
:103750000432A3503D493E4A3E4BD1603E49800071
:1037600019503E49E938FF3819503D490430195085
:103770003C491038D1613C4911633C4951633C4993
:1037800011603C49195019003B48F83108603B4929
:10379000D16582213A4A89005A501A0039490832C3
:1037A000D1671A003849B43211608821374A89003C
:1037B0005A501A00364988321160364ADA6408F0E5
:1037C0003FF9012008F0B4F970BD200014259C30A9
:1037D000056020000435A03070E7200010259C30E3
:1037E000056020000335A03068E720000E259C30DE
:1037F000056020000235A03060E7C0460004FF1FCE
:103800005C66FF1F5071FF1F1446FF1F4A0AFF1F0F
:103810003A07000080C3C9019A02000050C30000AB
:103820006A180000280A0000204E000088130000DB
:10383000F009FF1F001F001168100000C4090000FC
:10384000DC05000040420F0010270000FD1BFF1F99
:10385000FC00FF1F0000FF1F092FFF1F3132FF1F59
:10386000C930FF1FDD1FFF1FF91FFF1FA521FF1F0D
:10387000491FFF1FC928FF1F712CFF1FD918FF1FE9
:10388000D527FF1F3D25FF1F4925FF1F491EFF1F8D
:10389000011FFF1FC11DFF1FF7B50B0CFF270122E2
:1038A000009300233C001E001D009446019089B245
:1038B00062469A401000084018413618B6B2FF2FF1
:1038C00002D1012E00D19FB2009802401A41AD18DA
:1038D000ADB2FF2C02D1012D00D19CB20133102BCF
:1038E000E6D10320012E07D1012D04D1019B240133
:1038F000E4191C700138FEBD102EFCD10238102DC9
:10390000F9D00230F7E710B5064C2378002B07D129
:103910000548FFF7F1FD0548FFF7EEFD0123237091
:1039200010BDC0461D66FF1F3066FF1F2066FF1FCB
:10393000F0B58BB00D0001230190102936D8FFF7A8
:10394000E2FF00231A001B48C15C01335218102B00
:10395000FAD1023B002A29D0174B184C1F680023CC
:1039600006A9E25C1600FA5C56405E540133102B47
:10397000F7D102AA07F0ACFE2A0002A9019808F0CC
:10398000B7F807F0ADFE23681B18236007F0A8FE08
:1039900063681B18636007F0A3FEA3681B18A3608D
:1039A00007F09EFEE3681B18E360002318000BB0CD
:1039B000F0BDC0463066FF1FB444FF1F2066FF1FE6
:1039C0000223F0B501245C4D5C4E2B705C4B91B032
:1039D0001C705C4F039333682000BB7006F034FC0E
:1039E0000023984205D0BA78552A02D0332A00D055
:1039F00096E03360002006F095FE08F071F8FFF7BE
:103A00009FFD07F0CDFE1F22012400214E4B3626DC
:103A10001A704E4B1C704E4B19704E4B19689143E7
:103A2000163A0A431A60602219689143403A0A43E1
:103A30001A6007F085FE08F00BF8C120FF21464B05
:103A400080001A588A431A50C52292009858884319
:103A5000BF39014399509858404908408021C90115
:103A60000143802099509958C0050902090A014371
:103A7000995080213A48490107F00AFE03232200A9
:103A8000009338490194384808F0FAF82E22374953
:103A900004A807F0A5FE02AB04ACF6186178207804
:103AA000023406F0F1FBA642F8D1314B314A1968D5
:103AB00003201140A022D2020A431A608022196812
:103AC00092040A431A6019682B4A1140802292031B
:103AD0000A431A60294B2A4A934200D8012008F071
:103AE0007FF807F0DDFF07F043FE287807F0E8FDD8
:103AF000039B1878C0B208F0F3F807F029FF2149BA
:103B0000042007F0E5FE06F0D9FD00F0B1F800F062
:103B1000FBFD00F08DFE00F01BFA002011B0F0BD9F
:103B200000932100174A042008F09AF88023DB054F
:103B30009C62FFF78BFC5DE74A0AFF1F34F00040F0
:103B40001446FF1FB063FF1F480AFF1F490AFF1FEB
:103B5000680AFF1FBCF0004000E100E0FF00FFFF2B
:103B60001846FF1F9C58FF1F1856FF1F20BD00114D
:103B700014F00040FF7FF8FFFFFF9FFF5071FF1F11
:103B80000080FF1F3B00010870B5002529492A4A23
:103B90002A484D6308CA1B051B0DED188242F9D156
:103BA0000022274B8B63274B08211A628022264B69
:103BB0009205DA67254BDA688A43DA60244A12787C
:103BC000012A03D09A6823490A409A6002202249B8
:103BD000EE240A68E40082430A600121DA686C433B
:103BE0008A43DA600F3007F08BFF112007F0B8FE30
:103BF000112007F0C5FD194A200C040064239042EF
:103C00000AD8FA220023D200904205D9144B0A2187
:103C1000C01807F0D5FFC3B2124A1372124BD480FA
:103C20001B78002B04D1114B1021187807F038FEB7
:103C300070BDC046000005400806054080060540EE
:103C4000FF01000000F0004004E100E03CF0004013
:103C50004A0AFF1FFFDFFFFF00380040B70B0000DC
:103C600030F8FFFF9863FF1FD465FF1FD063FF1F6D
:103C7000002210B51100112007F05AFE10BD0000FF
:103C8000F8B5002301250826394F3A4C3B62E3681A
:103C90001120AB43E360E368B343E36007F060FEE9
:103CA000112007F02DFF112007F012FF402322689A
:103CB00029001343236080236268DB02134363609F
:103CC0008023A26830001343A360A3682A4A1340EC
:103CD000A3608023A2689B0113431022A360236C7E
:103CE00093432364236C2B43236480231B013B6297
:103CF000226B224B10271A402263626B1A406263C8
:103D0000A26B1A40A263E26B1340E3631C4AE368B0
:103D10001340E36006F09EFB2900300006F0C8FB6C
:103D20008023184A5B00516C11200B43536407F049
:103D3000CFFFFD21C720144B144A89005A50A36BB2
:103D400080003B43A363E368114A1E43E660E368D7
:103D50001D43104BE56019581140802212020A439E
:103D60001A50802292051A600B4B5F63F8BDC04663
:103D700000F000403CF00040FFFFDFFFEFFFEFFFEF
:103D8000FFFF7FFF003800400000FF1F893B00114C
:103D9000FF00FFFF00E100E00000054030B503A890
:103DA00004880B20002C0ED14968074D087849780B
:103DB000090201430A20A94205D1012120001980EE
:103DC000024B1B7A137030BD192A00009863FF1F45
:103DD000F7B5150008AA16884A680F4F147852786C
:103DE000120222430A24BA4214D10122DBB2019208
:103DF00000962A0007F0B2FB041E0BD1074B1B688C
:103E0000002B07D068782A780002104342425041C4
:103E1000013098472000FEBD022900001C63FF1FEF
:103E200030B5012503790400BFB02B4212D00A49F6
:103E3000408806F0FFFE28420CD06A46074B6946D0
:103E40005B8D55801380064B60881B7A13710022AE
:103E500003F0E2FF3FB030BD1463FF1F4842FF1F75
:103E60009863FF1F10B50549054806F099FE042127
:103E7000044A054806F056FE10BDC0461463FF1FF5
:103E8000FFFF000050BD00114842FF1F10B502485F
:103E900004F044FE10BDC046213E0011062310B5BB
:103EA000837010330371443B43712A33837144336D
:103EB000C37100230222012103720E4B0270417074
:103EC0001C8881724472197A0273C1729A784273A3
:103ED000DA7882730322C2731A7902745A794274AF
:103EE0000C2282749A79C274DB7903751123C37032
:103EF000152010BD9863FF1F10B5142007F020FD9A
:103F0000124B14220021186007F05AFC002007F021
:103F1000AFFB012007F08CFD022007F029FD0320F4
:103F200004F0A0F8042006F0B5F8052003F0DEFA4E
:103F3000062003F0ABFF072001F0A6F9082006F0E9
:103F4000D1FD092000F08EFF10BDC0462063FF1F89
:103F500010B507F04DFC012007F05AFE07F0B0FE47
:103F6000002010BD094B10B50400984205D001296E
:103F700004D12000064906F013FE10BD0229FCD131
:103F8000013904F089FD0028F3D0F6E7FEFF0000B8
:103F90004663FF1F70B50D7A100004AA2C00168826
:103FA00010221440154220D1002E20D10A78022A76
:103FB00018D14A68517815780E4A0902294391426E
:103FC00005D00D4A914209D01C800A2404E0142235
:103FD0000A491A8007F004FC200070BD0C22084931
:103FE0001A80F7E71C800124F6E70824F4E70B2485
:103FF000F2E7C046F3FF0000F4FF00009844FF1F03
:104000002CBE001110B504000749084806F0C8FD91
:10401000074804F0C3FC0020E40704D50721054A43
:10402000054806F07FFD10BD4663FF1FFFFF00003F
:10403000653F001194BD00118C42FF1F00B50C4B71
:10404000BFB01A780B4901A800F024FC6B4680B27F
:104050005880002809D06A46074B69461B881380A0
:10406000064B0022188803F0D7FE3FB000BDC046C3
:104070002463FF1F2563FF1FE642FF1FEE43FF1F60
:1040800000B50C4BBFB01A780B4901A801F00AFE2D
:104090006B4680B25880002809D06A46074B6946B3
:1040A0005B8D1380064B0022188803F0B5FE3FB0ED
:1040B00000BDC0464E63FF1F4F63FF1F8C42FF1FB2
:1040C000EE43FF1FF7B50E00377A1C0008AB110056
:1040D0003D001A8820231D401F423CD13378022B1B
:1040E0003BD173681F785B781B023B431E4FBB427A
:1040F00008D01E4FBB4214D01D4DAB4221D00A2523
:104100002800FEBD002A2AD1142C2AD82200F068EB
:1041100007F066FB174B1C70012CF1D9FFF7B0FFBD
:10412000EEE7002A1BD1202C1BD82200F06807F0F4
:1041300057FB114B04211C70104B187807F0B0FB93
:10414000DEE7E3B20124009201940A00310007F097
:1041500005FA0500D4E70825D2E70125D0E70B25AD
:10416000CEE70D25CCE7C046F3FF0000F4FF0000CA
:10417000022900004E63FF1F2463FF1FD063FF1F4F
:10418000332310B5040003700A220749013007F0F9
:1041900027FB064B0F201B681A0AE37222731A0CC6
:1041A0001B0E6273A37310BD9863FF1FC063FF1FD4
:1041B00030B5012503790400BFB02B4213D00B4961
:1041C000408806F037FD28420DD06A46084B01A80A
:1041D0001B881380FFF7D4FF6B4658800022694686
:1041E000608803F019FE3FB030BDC0464663FF1F34
:1041F000E642FF1F10B5024804F090FC10BDC04617
:10420000B141001170B5160004AA148805AA1578EA
:104210004A685078117800022A4A08438018052815
:104220004BD807F005FD03131E29343F0720032C4C
:104230000BD80422121BAA4200D92A0022491A8054
:104240003000091907F0CCFA002070BD0720112CAE
:10425000FBD81222121BAA4200D92A001B491A803D
:10426000EEE707200E2CF0D80F22121BAA4200D92D
:104270002A0017491A80E3E70720032CE5D8042217
:10428000121BAA4200D92A0012491A80D8E7072037
:10429000032CDAD80422121BAA4200D92A000E49A4
:1042A0001A80CDE70720032CCFD80422121BAA4284
:1042B00000D92A0009491A80C2E700220A201A8080
:1042C000C3E7C046DCD5FFFFDFBD00116C63FF1FF5
:1042D000CFBD0011CABD0011C5BD0011C0BD001188
:1042E00010B50D21024A034806F01CFC10BDC04663
:1042F000B4BD0011FC42FF1FF0B50024274E85B06D
:104300003000B47100F0E2F8254D264BEA89297C93
:104310009A422FD10423300003AA00F057F9040079
:10432000300000F011F90123B371002C34D16B4639
:1043300099892B68C9BA4B4329891B4A1B145B18FE
:1043400053806B46D9896B6849BA89B24B436989F6
:104350001B0C5B181548191C1BB2834200DD011CA5
:104360000B0400D5002113889180013313802000B5
:1043700005B0F0BD0227220003AB3000009700F02B
:10438000F7F80E230400297C0122300000976B44CB
:1043900000F0EEF80443C3E71C00E8E7D443FF1F36
:1043A0008063FF1F830500009863FF1F0F27000035
:1043B00073B5234E300000F089F8224D07236A467A
:1043C0003000297C00F002F904003000002C33D1C9
:1043D0006B461B787F2B2FD800F0B6F86B46D87849
:1043E000F02302041B031A406B469B8816495BBAF4
:1043F0009BB21A432B68000953432A891B0C9B1854
:104400004B806B465A789B7812031B011A436B68EA
:10441000024353436A891B0C9B180C481A1C1BB29D
:10442000834200DD021C130400D500220B888A8021
:1044300001330B80200076BD00F086F80124F9E7F7
:10444000D443FF1F8063FF1F9863FF1F0F270000E7
:1044500070B5114C237C002B0FD0382B0ED10F4D93
:10446000280000F033F8CC23AC222800217C9B01EB
:1044700000F0F4F8280000F067F870BD084BE289FE
:104480009A42FAD1054D280000F020F800222800B9
:10449000217C00F0C5F8EDE78063FF1FD443FF1FC8
:1044A0008305000010B5084B1A7C002A09D05B690F
:1044B000002B06D09847041E01D0FEF7A1FD200076
:1044C00010BD0124F9E7C0468063FF1F70B5C179B4
:1044D00005000C00631E9C411A4BE402E4184900DD
:1044E0000460C9B2007906F019F8E97968794900E1
:1044F0000131C9B206F012F8E8790930C0B207F00C
:10450000E7FA0023E36661332360AA795B3B002A64
:104510000ED022689A43023B134323600A23E361CF
:104520000733236200232363A3630133E36370BD76
:1045300022689A43022313432360462363610633B0
:10454000A361EFE70050004070B500250400036848
:10455000DD66C0790930C0B207F002FA290020797F
:1045600005F078FF2900607905F074FF70BD000048
:10457000F8B51E0006AB1D78002304681700E3663B
:10458000616007F0C5FA01238022E3662B002761F2
:104590005200013B08D207F0E3F808200A4A1168EC
:1045A000002D03D12800F8BD2261F2E7236F0342FA
:1045B00003D02369013D3370013613685B1A032B66
:1045C000EED90125EEE7C0466008FF1F70B51C005C
:1045D000002305681600EB66696007F099FA01236D
:1045E0008022EB6623005200013B08D207F0B8F8A6
:1045F00008200A4A1168002C03D1200070BD2A61EE
:10460000F2E72B6F034203D02B69013C3370013674
:1046100013685B1A032BEED90124EEE76008FF1F35
:10462000002370B504681500E366616007F070FA56
:104630000123E366256107F093F88020064A800095
:104640001168636B034205D113685B1A032BF8D919
:10465000012070BD0020FCE76008FF1F70B51D0041
:10466000002304681600E366616007F051FA012335
:10467000E36626610F33626B1A42FCD02B0A23617A
:104680001023626B1A42FCD0EDB2256107F068F886
:104690008020074A80001168636B034205D11368CC
:1046A0005B1A032BF8D9012070BD0020FCE7C0463F
:1046B0006008FF1F70B51E00002305681400EB663C
:1046C000696007F025FA0123A619EB660F33B4429F
:1046D0000ED107F045F880200A4A800011686B6B04
:1046E00003420CD113685B1A032BF8D9012070BD6B
:1046F00021782961696B1942FCD00134E7E7002079
:10470000F5E7C0466008FF1F10B5084CE368002BB2
:1047100008D1074B1B685B045B0C0A336360054BD5
:104720001B68236007F0E4FAA06010BDC063FF1FA0
:10473000C8F00040CCF0004010B507F0E9F90F4B8D
:10474000996A9A6A8A42FBD10D4C6268A0688A18FD
:10475000121A531E884200D31300A1602168DA0B9D
:1047600052185B0407495B0C636022600B60064BC8
:104770001A6006F0F5FF206810BDC04600F000404A
:10478000C063FF1FC8F00040CCF0004070B51F4C64
:1047900023793F2B01D93F2323711D4B22791A70B6
:1047A0001878C0B207F0ECF918231A491A4A0B809E
:1047B0001A4913800B805380A379194980200B80FC
:1047C0000C21938001334B430001191C834200D913
:1047D000011C144BD18019806379002B11D1013356
:1047E0006371237A012B01D8022323726279237A21
:1047F0000D4853430A21584307F0E2F90B4D286056
:1048000070BDA02BEDD9A023EAE7C046B463FF1F1B
:10481000480AFF1FEC43FF1FC045FF1FEA43FF1F6D
:10482000A065FF1FE843FF1F71020000A463FF1F84
:10483000F8B513210020FEF7D1FD114C011E114DDA
:1048400009D10C22104BC1CBC1C4280006F0B8FF1F
:10485000FFF79CFFF8BD0C2220000C49FEF792FDEB
:104860000C2802D0084B43CB43C40C222800084933
:10487000FEF788FD0C28EBD00C220021E5E7C046AE
:10488000B463FF1F8063FF1F20BE0011FC0C0000FB
:10489000F50C0000F0B5002504000E0085B0AA421A
:1048A00068D04B1C087801934B78897837790902D6
:1048B0001943F3783F061B040B431F4303972070F3
:1048C0006570262800D190E01CD8102812D807F077
:1048D0001FF84B0004013100310031009600A400A4
:1048E0009D003100310031003100310031003100D4
:1048F0003100E400232800D1BEE025285DD0FF234D
:10490000637099E0602800D1A1E00AD8552834D01E
:1049100056284CD03328F2D12000FFF731FC050097
:1049200028E0722800D189E0DC2800D1F4E0712869
:1049300000D179E0DB2800D009E1042ADFD9102575
:10494000052A05D0551F2A003800711D06F048FFC2
:1049500005223100200006F043FF2A003900601DC7
:1049600006F03EFF053505E00C2220008E4906F0DA
:1049700037FF0C25280005B0F0BD013A8B4D0C2AFD
:1049800013D8002A0AD02800019906F029FFFFF762
:10499000FDFE0C2228008649FEF72EFC29000C2281
:1049A000601C06F01DFF0D25E4E70C22EBE77F4DB0
:1049B000804B2A0043CB43C2E9E7013A7E4D0C2AE3
:1049C00011D8002A08D00199280006F009FF0C220E
:1049D00028007A49FEF710FC29001322601C06F01B
:1049E000FFFE1425C6E70C22EDE7734B29001322C6
:1049F00018001D0006F0E4FEFEF702FBECE70522BE
:104A00006F49601C06F0ECFE0625B3E712226D49E3
:104A1000601C06F0E5FE1325ACE708226A49601C1D
:104A200006F0DEFE0925A5E77178F72900D966E7CB
:104A3000664B188801F092FD02259BE7644B012A22
:104A400003D072785A706270F6E75B7858E7013AE3
:104A5000604D072A0ED8002A05D00199280006F0DB
:104A6000BFFE01F059F829000722601C06F0B8FECD
:104A700008257FE70722F0E7042A04D9564D2F6066
:104A800007F036F9A860FFF757FE0422039003A948
:104A9000601C06F0A5FE05256CE7504D062A15D9C9
:104AA00006222800019907F0CBF800280ED0062234
:104AB0000199280006F094FE062249492800FEF7D5
:104AC0009BFB0123424A51780B4353702900062275
:104AD000601C06F085FE07254CE7931E414F1A2BFC
:104AE00004D87378002B09D100F030F93E4B39001F
:104AF0001D78601C6A1E06F073FE3BE7551E2A00F7
:104B00000199380006F06CFE3849AAB23800FEF769
:104B100073FB00F051F9E9E7022A00D8EFE6737859
:104B2000BFB26370B378A370032A05D0033A39008B
:104B300092B2F01CFEF760FB10223900E01CFEF779
:104B400021FCC51C002800DB14E7607074E7DA283C
:104B50001DD1042A00D8D2E6082A15D9B379727972
:104B60001B021343F27912041A43337A1B061343D0
:104B70003B603B68052231002000039306F030FEC5
:104B80000422601D03A94BE7FE236370F1E7DE28D2
:104B900000D0B4E6511E012A01D10025EAE60198B1
:104BA00000F0A0FFF9E7C0462CBE0011B463FF1F60
:104BB000FC0C000020BE00118063FF1FF50C0000FC
:104BC0008C63FF1F6C63FF1F3445FF1FEE43FF1F05
:104BD000B063FF1F8944FF1FC063FF1F6509FF1FEC
:104BE000ADAC0000B365FF1FB165FF1FAEDE000076
:104BF00070477047020010B5094B0A32094C92B257
:104C0000DA815A8298811882207802F00DFB042202
:104C1000054B012120781A7006F042FE10BDC046F7
:104C2000BE44FF1FFE65FF1FFD65FF1F013870B505
:104C3000042809D806F0FCFF030928081200234BBA
:104C40000221187806F02CFE70BD204B0821187840
:104C500006F0AEFF00221E4B1A72F5E780220024F8
:104C60001B4B1A4D52001A8108211A682878DC72F1
:104C700006F096FF2100287806F0BAFF012000F028
:104C800051FE00F049FFDFE7104B0821187806F0CD
:104C90008FFF1048FFF702F90F4B104A9B79002055
:104CA00093800F4A13808022094B5200D8721A81D8
:104CB00000F038FE00F030FF0A4B5B78002BC3D0C9
:104CC000094A136006F084FDBEE7C046D063FF1FAB
:104CD000A463FF1FF743FF1FB463FF1FC045FF1FFF
:104CE000A065FF1FB063FF1F34F0004010B501291D
:104CF0000BD1012809D1054B1B78002B05D02622AA
:104D0000034B04485A72FFF775FF10BDD465FF1FAF
:104D1000A463FF1FC40900000300F0B50A4D8E18FC
:104D2000B14202D152008018F0BD0C782F682409DE
:104D30003C5D0F271C700C7801313C402F683C5DB6
:104D40005C700233ECE7C046E443FF1F0D22114BB9
:104D500010B51A700C23104C10492370093A033B0C
:104D60000F48637006F03CFD2D2301220D490E48CB
:104D7000A371FFF7D1FF01220C49FFF7CDFF0122FC
:104D80000B49FFF7C9FF00220A491000FEF734FA69
:104D900010BDC046D065FF1FB165FF1FDFBD00110C
:104DA000B365FF1F6709FF1FB865FF1F6609FF1F77
:104DB0006509FF1FAEDE000070B5124C1322200003
:104DC0001149FEF7DFFA114D002817DDAB78002BF3
:104DD00014D0431C2B7009236B700023001903703F
:104DE000287829000130C0B206F022FD297822007F
:104DF0000139C9B2002005F0B3FD70BDFFF7A6FF71
:104E0000EEE7C046B365FF1FAEDE0000B165FF1FD1
:104E100010B5114B1A781870002A0ED000280BD14B
:104E20000E4B1A78062A07D85423D340DB0703D544
:104E30000B4B187802F0F8F910BD0028FCD0074B96
:104E40001B78012B02D0033B022BF5D8044B012128
:104E5000187806F025FDEFE7D465FF1FFD65FF1FFD
:104E6000FE65FF1F70B54A4E4A4A4B49307001201B
:104E700005F002FC00F0B4FEFEF7C2F806F0C8FD33
:104E8000032246494648FFF747FF2D24030004222A
:104E90001C7044490130FFF73FFF30230470424D3E
:104EA000424C437083702E3B062220004049EB8722
:104EB000FEF768FA062813D0200006F0E1FB02286E
:104EC00009D00321200006F01BFD8D23E3706E3B0B
:104ED000237119336371062220003549FEF78CF9DE
:104EE000344B1B68FC335C64FFF766FF0020FFF760
:104EF0008FFF314C314A0121314B1278207802F07A
:104F000055F9304A304B12780021207802F04EF9E2
:104F100001222E4B1A702E4B9B78552B31D12D4BE5
:104F20003B325A722C4B2D4AAB81EA812B826A822A
:104F30002021307806F004FE0120404205F05CFD9F
:104F40000120404205F0F8FDFFF7CAF9FEF78AFF9D
:104F500000F0A6FC01204042FFF754F8012006F0C3
:104F600027FCF72001F0DEFA0121307806F098FCEA
:104F7000307802F0B5FA1A4806F09AFBFEF780FE88
:104F800070BD6422174B5B7953431A000A32CBE79A
:104F9000D063FF1FF14B0011ED4C00113445FF1F92
:104FA0006C63FF1F8C63FF1FBE44FF1F6509FF1F5B
:104FB000ADAC00005C66FF1FFE65FF1F1644FF1FBF
:104FC000F743FF1FD065FF1FB165FF1FA265FF1FDD
:104FD000B063FF1FA463FF1FC4090000CE090000D7
:104FE000D263FF1FB463FF1FF8B50A0020230D0032
:104FF0001A40194257D0574B1B78002B50D0FFF75F
:105000009BFB554B554C564E99686268737A8A1AC9
:10501000DB039A4202D36160FEF732FE327A217AD4
:10502000531EDBB2994205D1FFF712FA002000F0BF
:10503000A9FD0FE09142F9D300232372FFF732FA62
:10504000012000F09FFD474F3800FEF727FF390091
:1050500006F02EFE637A002B1FD0013BDBB2637299
:10506000002B1AD1404B9B78552B01D106F0B0FB99
:10507000E37A002B0CD000233C4A3A4FE3721388AA
:10508000380001331380FEF709FF390006F010FEE7
:10509000642370795843FFF7ADFD237A01332372FF
:1050A00020206840F8BD0BB2002B0ADA304B18788C
:1050B00006F0CEFD002801D006F05AFD8020000247
:1050C000EFE70224214206D0244B01201A72FFF799
:1050D0009FFE2000E5E70B071ED5FFF72DFB1E4BBB
:1050E0001E491F4C98684A68637A821ADB039A4209
:1050F00002D34860FEF7C4FDFFF7D4F9FFF7A8F923
:10510000012000F03FFD00F0E5FB2368DB0701D53F
:10511000FFF770F80820C4E71024214206D00D4B99
:105120001B78002BD5D1FEF7B1FED2E70124214236
:1051300007D0104800F06CF806F072FB00F008FD94
:10514000C7E70424080020402142ABD0FEF776FFD9
:10515000BFE7C046D465FF1FC063FF1FA463FF1FE6
:10516000B463FF1FF743FF1FB063FF1F9863FF1F68
:10517000D063FF1FDC43FF1FF0B51B4B1B4F1B8889
:105180003A8804001A4E1B4D85B09A420DD83288D9
:105190009A420AD3184B1A882B889A4205D1174A8B
:1051A000174B12881B889A421BD0052001F010FA79
:1051B0003B8802AA13803388019053802B88114DBD
:1051C00093800F4B02A91B88D3800F4B2A78188835
:1051D00002F02CFF0D4B08212878019A1C7006F074
:1051E00067FB05B0F0BDC0469E65FF1FEC43FF1F87
:1051F000EA43FF1FA065FF1F9C65FF1F9A65FF1F05
:10520000E843FF1FFE65FF1FEE43FF1F9865FF1F6A
:1052100013B50C4B1C78002C11D1002801D00A4B7F
:1052200018600A4A0A4B11780A4A10780A4A019211
:105230000A4A0092002205F08BFA200016BD1124C4
:10524000FBE7C046FD65FF1F9465FF1FFC65FF1F60
:10525000EC65FF1FFE65FF1FD865FF1FDC65FF1FA4
:1052600010B5064B12201B78052B06D1044B1322D8
:105270001988044B187801F087FB10BDFD65FF1FEE
:10528000EE43FF1FFE65FF1F10B500240122114BE6
:1052900052421870104B1C70104B1A8002F020F90B
:1052A00004220F4B21001A700E480C3206F028FD24
:1052B000102221000C4806F023FD07220B4B1C6036
:1052C0000B4B1C700B4B1C700B4B1A700B4B1C7058
:1052D00010BDC046FE65FF1FFD65FF1FEE43FF1FAB
:1052E000FC65FF1FEC65FF1FDC65FF1FD865FF1F16
:1052F000B065FF1FAF65FF1FF043FF1FAE65FF1FC7
:10530000F8B5174C0600257806A814240078052D5A
:1053100023D1B41F134FA5B21824BD421DD88D1F31
:10532000ADB2BD4219D8FA256D00AA4215D21D00B2
:105330000D4F0A3DADB2BD420FD80C4C26800C4C2F
:1053400021800C4900240A800B4A1380FFF714FFC8
:105350000A4B0421187806F02BFC2000F8BDC0464B
:10536000FD65FF1F790C0000750C0000EC43FF1F6A
:10537000EA43FF1FA065FF1FE843FF1FFE65FF1FF5
:10538000F0B50BB20D0089B0002B00DB70E1A44E2C
:10539000307806F05DFC041E50D00378A22B00D1BB
:1053A00022E1D02B1AD0912B45D143780E2B42D13C
:1053B0009C4B82889A423ED19B4A83681278052A88
:1053C00039D1032018567F2835D0984B1B68002B05
:1053D00031D05B68002B2ED098472CE080780728CE
:1053E00029D806F025FC0428183F3F74A8D8637814
:1053F000002B0CD101218C4B19708D4B1A78002A8F
:105400005BD08C4B307801F0D1FE002855D00722BC
:10541000854B1A7051E061780029F8D1E378002BB0
:1054200011D0854A854B1278307801F0BFFE60704C
:105430006378002BEBD1200006F09AFB802000025D
:10544000684009B0F0BD784B1B78022BF3D00121E6
:10545000307806F0E5FA0028EAD10121307806F02C
:105460001FFAE5E76378002BD1D16F4F032807D1EE
:105470003B78052B02D101333B701EE00223FBE792
:105480006F4B1A886F4B0293002A0BD01B78002BAE
:1054900003D00121307806F00BFA3B78062B04D1BB
:1054A000013BE9E7029B1A70F7E7042B41D1012188
:1054B000029B3078197006F0F3F95C4B1B68002BE7
:1054C000B9D01B68002BB6D0574A107884E76378B0
:1054D000554F002B27D10622211D5B4806F080F98D
:1054E00062895A4B5A491A80A2895A4B1A80E38919
:1054F0000B800521397058490A80584A1380228A46
:10550000574B1A80574B1B78012B09D11F2001F0F4
:105510005FF8FA22920042430421307806F0C8F97D
:105520000022484B75E7312B00D070E70022454B35
:105530001A700323A0E706220021434806F0E0FB8F
:105540000023454A04211380444A30781380444A9A
:10555000138006F02DFB0821307806F029FBA37993
:10556000083B5A425341304A03331370304B1B7887
:10557000002B06D0334B30781A78002A06D001F081
:1055800053FE0122314B52421A8096E701211970D5
:1055900006F086F9F5E70821307806F009FB637814
:1055A000002B00D047E72C4B2D4F0293E388029A43
:1055B00004211380294B307803932389039A1380A5
:1055C00063893B8006F02CFA002800D033E7264B95
:1055D0001B68002B00D12EE7039902983A880988AE
:1055E00000881B68984726E74379132B00D022E7F1
:1055F0000389012B0AD11D4B1B78022B06D10821F0
:10560000307806F0D5FAFFF72BFE14E7052000F0FE
:10561000DFFF08210200307806F04AF90BE7C046A8
:10562000FE65FF1F05140000FD65FF1F9465FF1F49
:105630001644FF1FF743FF1FD065FF1FB165FF1F13
:10564000D265FF1FD465FF1FA365FF1FEE43FF1F39
:10565000AA65FF1FAC65FF1F9E65FF1F9C65FF1FAE
:105660009A65FF1FA265FF1F9065FF1F9865FF1FCA
:105670008020C001014200D0E2E6CB0731D5324B99
:105680001B78002B1DD0314E05AC3378052B1AD179
:10569000023B23702E4B21001B7823722D4B1B786D
:1056A00063722D4B187801F025FD002809D00720E2
:1056B0002A4B30701B68002B03D01B68002B00D0D6
:1056C00098470120BCE60E20254B06221B78254971
:1056D0002370254B1B78637002ABC01806F080F86E
:1056E000D8E7022308001840194209D0174B1B784D
:1056F000052B03D11D4B188806F04AFA02209FE6BD
:105700000424214203D0FFF737FD200098E6082348
:1057100008001840194200D193E6154B1C78012C63
:1057200003D0022C0DD008208AE6124B124A1349EE
:1057300013481B881288098800880094FFF7E0FD51
:10574000F1E7FFF78DFDEEE7D465FF1FFD65FF1F55
:10575000F043FF1FAE65FF1FFE65FF1F9465FF1F2F
:10576000B065FF1FF143FF1FAF65FF1FEE43FF1F33
:105770009865FF1FE843FF1FA065FF1FEA43FF1F57
:10578000EC43FF1F10B502A804880B20002C10D199
:10579000496808784978090201430C48814209D1D7
:1057A000022119800A4B59881170DB7800205BB206
:1057B000537010BD074C0A20A142FAD10221198072
:1057C000034B998811705B79F0E7C0466E2A0000A0
:1057D0009863FF1F6F2A0000F7B5150008AA168806
:1057E0004A680F4F14785278120222430A24BA42B0
:1057F00014D10122DBB2019200962A0005F0AEFE20
:10580000041E0BD1074B1B68002B07D068782A7841
:105810000002104342425041013098472000FEBD33
:10582000022900001066FF1F30B50125037904002E
:10583000BFB02B4227D01549408805F0FBF928421C
:105840000DD06A46124B69465B8D1380022353804C
:10585000104B5B8893806088002202F0DDFA0E49CD
:10586000608805F0E7F9C0070DD56A460B4B69461D
:105870001B88138002235380064B9B88938060888B
:10588000002202F0C9FA3FB030BDC0460866FF1FD3
:105890001844FF1F9863FF1F0066FF1F7244FF1F1D
:1058A00010B5074C0749200005F07AF92000064999
:1058B00005F076F90721054A054805F033F910BDD2
:1058C000FFFF00000866FF1F0066FF1FACBE00114F
:1058D0001844FF1F10B5024803F020F910BDC04660
:1058E000295800110221430888400B400A31084022
:1058F00003430E20024AD17881430B43D370704793
:105900008944FF1F064A1379410705D580210B43BF
:1059100080011371907170477F210B40F8E7C046FA
:105920008944FF1F054A5378002803D080210B4388
:10593000537070477F210B40FAE7C0468944FF1F30
:105940000F21114BDA780A40DA70502810D9013152
:105950000A43DA702022D9780A43DA704022D978D3
:105960000A43DA708022D97852420A43DA7005E09D
:105970003C28EFD82828F1D81428F3D80122D97868
:105980000A43DA707047C0468944FF1FF8B57F2389
:10599000324D04006E789E43314B984205DD7623EC
:1059A0002B70363B33436B70F8BD2E4B984203DAB5
:1059B00058232B701433F5E783B21A0000215F32AD
:1059C000294892B2294F297082422DD9A9708C4260
:1059D00003DA5B421CB220232B70053420B20A216B
:1059E00006F0EEF804B2FA239B009C4233DB8023DE
:1059F0002A785B4213432B706421200006F0E0F804
:105A00000A2100B205F0FCFF09B22A787B5C13433F
:105A10002B700A21200006F0D3F80A2100B205F00D
:105A2000EFFF09B27B5C0AE08022AA70002CDADA70
:105A30005B421CB220232B705F23092CE9DC1E4340
:105A40000A2120006E7005F0DBFF09B2AA787B5CAA
:105A50001343AB70A8E7632CCEDCEDE78944FF1F4E
:105A60001B4E00001DFCFFFF2A080000D6BE0011DF
:105A70007F23F7B5194FCD013E7904009E433E7157
:105A8000EDB2632806DD093B33433B7140231D43E0
:105A90007D71F7BD0300093304DA582333433B71AA
:105AA0006C23F4E70E4B019300280BDA04234442E5
:105AB00024B23B710A21200005F0A2FF019B09B22C
:105AC0005B5CE4E70928F5DD0A2106F079F8019B23
:105AD00000B21B5C1E433E71ECE7C0468944FF1FC9
:105AE000D6BE0011F8B50A4F05003B780E00002B1A
:105AF0000CD0084C2000FEF7E9FC33002A002000FF
:105B00003978FEF7D7FD2000FEF71EFDF8BDC04630
:105B10001C66FF1F9044FF1F70B50A4E0A4D0722F6
:105B20003100280006F08CF8002809D0074C31001D
:105B30000722280005F054FE08212000FFF7D2FFBD
:105B400070BDC0468944FF1F1566FF1F1466FF1F06
:105B50007F2210B50A4B59789143033A1A70103AD4
:105B60000A435A7078220E219A70DA788A43DA70E2
:105B700006221A7129325A71FFF7CEFF10BDC046B6
:105B80008944FF1F10B5002824D0134C0A2102239A
:105B9000E05E06F015F800B2FFF7F8FE0423E05EC1
:105BA000642106F00DF8012100B2FFF761FF207AB1
:105BB000FFF7C6FE0320FFF795FE0020FFF7A2FEC9
:105BC000064B1878053843425841C0B2FFF7AAFE89
:105BD000FFF7A2FF10BDC0469863FF1FFD65FF1FC2
:105BE00070B50024094D2800AC71FEF76FFC10233E
:105BF0003E212800064AFEF75DFDA04200D13E345A
:105C0000044B28001C70FEF79FFC70BD9044FF1FE2
:105C1000C6BE00111C66FF1F0200F0B501270A482E
:105C20000A4E51188B1A002B00DCF0BD08241578A1
:105C30004308684038404000805B013C58406D0894
:105C4000002CF5D10132EDE7FFFF0000E6BE0011A8
:105C5000F0B500250F269D4200DBF0BD4C5D070925
:105C600044403440A400A05801357840F3E70000D8
:105C7000F0B589B06A460D000B000F2711001035F2
:105C80001C780133260024093E40167054700232FD
:105C9000AB42F5D12023024AFFF7DAFF09B0F0BD8D
:105CA000ECBE0011F0B54E780B7889B036020C00CE
:105CB000170001901E43012A61D9954B9E4200D8DE
:105CC00077E001339E421CD1062A17D1CA788B781F
:105CD00012021A430B791B0413434A7912061A4322
:105CE0008C4B5A6100221A705A808B4A5A608B4A38
:105CF0009A608B4ADA60002009B0F0BD8822520514
:105D0000EEE7884B9E423CD182498B78002B00D035
:105D1000F6E00C2A31D10F22A3789343E2781202E5
:105D200013432279120413436279120613434B6022
:105D3000E279A07912020243207A00041043627AC9
:105D400012060243CA60E27AA07A1202024376483F
:105D50004A81834208D804236E49142201980B70AB
:105D600005F03EFD1420C7E71201D21889235B0518
:105D70009A42F0D801238B70BDE7022AFAD005239E
:105D8000EAE76A4A01239642E6D1FFF769FA052F4E
:105D90000CD9E378A2781B021343227912041A4328
:105DA00063791B061343624A0393136005F010FDE9
:105DB000A1E7584D2B78002B9DD1AB78002B00D15B
:105DC000A0E02B8901339BB20093B34200D091E055
:105DD000132AD4D9CF7C8B7C3F02122120001F4391
:105DE000FFF71AFF874200D08EE0002E3DD1E37806
:105DF000A2781B0213432279E96812041A436379DB
:105E00001B06134303930A228B4212D1FF23A37074
:105E1000E370237163716B89002B09D1E37B227CD2
:105E20001B0212041343A27B13431B0901336B8132
:105E300000226B89002B8ED0002A67D16868370159
:105E40003818000B6B6900030390984205D968610C
:105E500005F0D6FCEB780133EB7068681022A11CCA
:105E6000381805F00DFD2E8145E76F89009A7B1EDD
:105E70009BB293423AD1E278A37812021A43237973
:105E800005A81B04134362796C6812061A43EB6879
:105E900000920392211D0C22049305F0A1FC012025
:105EA000260004A940421036FFF7E2FE013F012F11
:105EB00017D1009A0B232861824200D04CE70422BC
:105EC0001C49200005F0DCFC042203A9686805F0E9
:105ED0007FFDE968039AFF23914200D13CE7F73B3D
:105EE0003AE73100FFF7C4FE1036DFE70923B74277
:105EF000A4D831E7009BB34200D9FCE607232BE787
:105F0000022329E7032327E7062325E70A2323E7BC
:105F1000FFFE00009844FF1F00000111FFFF00007A
:105F20005048593601FF0000FFFF001102FF00003A
:105F300034F00040A444FF1F10B5034C0B000122B5
:105F4000210000F06BFA10BDF96000110B8870B5EC
:105F500006000D000224162B11D92B00032209493B
:105F600000F05CFA041E0AD1074B2A881B88191C12
:105F7000934200D9111C300089B200F0EFFA2000E2
:105F800070BDC046256100117666FF1F10B54A78C6
:105F90000400013A0B000220012A07D80A78002ADF
:105FA00004D005222000024900F038FA10BDC04696
:105FB000536100110A7810B50B0004000220002A7A
:105FC00004D007222000024900F028FA10BDC04684
:105FD000FF6100110A7810B50B0004000220002AAE
:105FE00004D009222000024900F018FA10BDC04672
:105FF0006562001110B5034C0B000B22210000F06C
:106000000DFA10BD9562001110B5034C0B000D2266
:10601000210000F003FA10BD0763001110B5034C16
:106020000B000F22210000F0F9F910BD616300118F
:106030000A7810B50B0004000220002A04D01122B7
:106040002000024900F0EAF910BDC046716300115A
:10605000002310B51322190000F0E0F910BD000074
:1060600010B5034C0B001722210000F0D7F910BD2A
:10607000C3630011002310B51922190000F0CEF9F6
:1060800010BD000010B5034C0B001B22210000F0D6
:10609000C5F910BDFD630011F7B584890D00060038
:1060A0000121002C22D000238268D3561778002BC0
:1060B0001EDA0C2C1AD90C3CA4B213194088009398
:1060C000230002F086FE431E984101307B06DB0F61
:1060D0006B703F23013C1F40A4B22870AF70AC80AE
:1060E000002C07D0B3680133AB6000210800FEBD6F
:1060F0000020EBE7AC60F8E70B7803704B88437047
:106100004B881B0A83700B79C370042070470420EE
:10611000022B06D10020537811781B02009A0B4302
:10612000138070470B8803700B881B0A4370022092
:1061300070470420009983420AD1537810781B02DB
:1061400003430B80D37890781B02034300204B80DD
:106150007047F8B50D004B7801240021461C0370F0
:106160002B788B4201D82000F8BD6B78B01C4F1CF7
:10617000012B10D1890069184B88022233704B889B
:10618000B9001B0A7370691805F0B2FC04360434B8
:10619000A4B2F9B2E4E7122359436B185A880431C8
:1061A00032705B8810221B0A7370691805F0A0FC1E
:1061B00012361234ECE770B5049D14001E00052B56
:1061C00001D8042070BD637812781B0213432B8022
:1061D000E378A2781B02134302226B802A71211DEF
:1061E000681D063E05F084FCB2B22A81F02AE8D888
:1061F0002800A11D0A3005F07BFC0020E2E7002307
:1062000010B50A789A4201D8900010BD9A008A18F9
:106210005488013304705488DBB2240A4470948893
:1062200084709288120AC2700430EAE710B5110037
:10623000029C062B04D004201022142B01D010BD88
:10624000022222714B7808781B0203432380CB780B
:1062500088781B02034363800431601D05F048FC0D
:106260000020ECE710B50C788B7804315C43E4B285
:1062700003702200013005F03BFC601C10BD0420BF
:10628000022B06D10020537811781B02009A0B4391
:106290001380704710B50C000A88023105F028FC05
:1062A000208810BD70B504000D0004981100012B6A
:1062B00001D8042070BD1678527812023243028051
:1062C0000200F83255701470E825002C00D10C350E
:1062D000023B9AB24280AA42EBD80231043005F068
:1062E00007FC0020E6E70420009983420AD1537896
:1062F00010781B0203430B80D37890781B02034372
:1063000000204B80704710B50C000A88023105F060
:10631000EFFB208810BD000070B501211E00042095
:10632000049C0E400B4218D1CB40DDB28D4214D9F3
:106330000A49DBB2098899420FD32300F6331D7056
:106340003300580011184978165C090231430133B3
:106350002152D9B28D42F4D8002070BDB844FF1F3D
:1063600010B50C000A88023105F0C2FB208810BD70
:1063700010B50C788B7804315C43E4B203702200D2
:10638000013005F0B5FB601C10BD10B5110002987E
:10639000032B01D8042010BD14785278043B12025C
:1063A00022430280CA788C781202224342809AB239
:1063B0008280F22AEED80431063005F099FB0020E5
:1063C000E9E710B50C000B8803700B881B0A4370BB
:1063D0004B8883704B881B0AC3708A88043006314F
:1063E00005F086FBA088043080B210BD0420012B8C
:1063F00003D100201378009A1370704710B50C0079
:106400000B8803700B881B0A43704A8802300431E2
:1064100005F06EFB6088023080B210BDF0B589B027
:1064200003931E4B029242000700D05A019102F0E2
:1064300020F81325061E2DD0029B01240370019B1A
:10644000002B04D0001903999847001984B26B46B9
:106450001B7A5BB2002B0FDA1021380002F01CFB14
:106460001925002813D130003219E1B202F066FC80
:10647000051E0CD10C34A4B2042304AA380005A9CB
:1064800093800696948101F0AFFD051E02D0300086
:1064900005F0D6F9280009B0F0BDC0467466FF1FAC
:1064A00070B505000C0000280CD00020814209D0F6
:1064B00010222000044905F01BFB01202B782373D8
:1064C0006B78637370BDC0462CBF0011F0B5060039
:1064D0000D0017001C0085B002291BD000201029D8
:1064E00007D1022B07D0102B03D115E00020102C70
:1064F00008D005B0F0BD69463800FFF7D1FF2A008B
:1065000069460BE069463000FFF7CAFF2200694682
:10651000380004E0022BE9D12A003900300005F0F0
:1065200077F9E6E7031CF72800D9F7230320084989
:106530009AB2013A0B80D317034006499B189B106F
:106540000B80D30F04499B185B100B807047C0462B
:10655000BC44FF1FBA44FF1FB844FF1F034B1B88F6
:106560008B4202D3024B4000C1527047BC44FF1F14
:106570007466FF1F014B4000185A70477466FF1F76
:106580001722014B1A8070477466FF1F70B5050013
:106590000E2005F045FB041E13D0D023037000230A
:1065A0000622837007494570033005F0A1FA064BB7
:1065B0002100DA8A62811B7E2373044B187805F070
:1065C00057FA70BD9066FF1F8066FF1F0C45FF1FC6
:1065D000262803D8024B4000C05A70470148FCE708
:1065E000BE44FF1FFFFF000070B506000C00094D00
:1065F0001C220021280005F083FB074B1E70074B6F
:106600001C7005F025F90123002801D00023122079
:106610002B7070BD8066FF1F0C45FF1FA166FF1F1A
:1066200070B505000D4C0800E260A1601022002149
:10663000656005F015F9012803D11021A06802F06A
:1066400058FD10220021280005F00AF9012803D185
:106650001021606802F04DFD70BDC0468066FF1FCE
:1066600070B5041E05D1002903D006220D4805F09F
:106670003FFA0D4B1D78012D11D1002C05D10222BE
:106680001A7005F02DF9280070BD00221A70074B12
:106690001B78FF2BF7D02000FFF778FFF3E70025EA
:1066A000F1E7C0469066FF1F8066FF1F0C45FF1F85
:1066B000030010B5002801D1002010BD00780B4A5E
:1066C000002803D15988D1821B7913761378022BC5
:1066D000F2D10023984200D103331370044B1B788E
:1066E000FF2B01D0FFF752FF0120E6E78066FF1F76
:1066F0000C45FF1F002911D000280CD04B79012830
:1067000003D140225242134303E03F2213400328A7
:1067100002D001204B7170474022F4E70800FAE7ED
:1067200070B5094D0100287800280BD0074C0622CF
:10673000200005F0DDF921002878FFF7DBFF2000BD
:1067400004F0EEFF70BDC046A066FF1F7A66FF1F13
:1067500000290AD0012808D13F224B799343C02B4E
:1067600003D0403B5A425341981C704770B5174DB7
:1067700006002B78FF2B15D00A2005F051FA041ED5
:1067800010D0D0230370C83B8370114B11491B7884
:106790004670C3700622043005F0AAF9210028785B
:1067A00005F066F90C4B1B78012B0DD10B4B1B68C8
:1067B000002B03D09B68002B00D09847084B042186
:1067C0001878084A05F0ECF970BDC0460C45FF1F6B
:1067D000A066FF1F7A66FF1F9C66FF1FC866FF1F2B
:1067E000CC66FF1F60EA0000014B98687047C04606
:1067F0008066FF1F014BDB68186870478066FF1FCB
:10680000074B10B5DA68136801331360054B18782D
:10681000FF2803D08021C90105F042F810BDC04611
:106820008066FF1F0C45FF1FF7B50E0002F0C8F889
:10683000051E1CD00E4B06621F78002F00D1077872
:10684000AB791020019305F0EBF9041E0FD0D02393
:106850000380C73B8370019BE91DC370062204308F
:1068600005F046F921003800E66005F001F9F7BDB2
:106870000A45FF1F014B18787047C046A066FF1FEE
:10688000054B002805D1054B1A78054B002A00D18D
:10689000014B18007047C0469066FF1FA066FF1F9F
:1068A0007A66FF1F014B58687047C0468066FF1F1D
:1068B000024B1868431E9841C0B27047A466FF1F80
:1068C000421E03000120152A03D9FF3B5A425341BF
:1068D000D8B27047F0B51C0000230E0085B00390BD
:1068E00002920B70029A934201D3002019E0E55CFA
:1068F0005A1CD2B2002DF8D0029851198142F4DC12
:106900000233DFB2A35C18000193FFF7D9FF002820
:1069100007D0013D019A0399EBB233708A4202D14C
:10692000E01905B0F0BDDB19DBB2DBE710B50C00F8
:1069300002F09EF803001220002B03D0210058889B
:1069400005F056F810BD000070B50E4D8400635977
:10695000002B15D0186A002801D004F0B1FF2B5984
:10696000586A002801D004F0ABFF2B59986A002820
:1069700001D004F0A5FF285904F0A2FF00232B51F9
:1069800070BDC046B066FF1F1C4B70B504000E0002
:10699000150099420AD11A4B1B68002B01D1122015
:1069A00070BD1B68002BFAD09847F9E7154B994248
:1069B00015D1134B1B68002B0AD01B68002B07D086
:1069C0009847002804D1104B1C70104B1D70E7E74E
:1069D00029002000FFF7AAFF0028E1D1F3E7080013
:1069E00001F0EEFF0028DAD003780320A342D7D1CC
:1069F0002900300004F0FCFFD2E7C046FEFF000093
:106A0000AC66FF1FFFFF0000A966FF1FA866FF1FFF
:106A1000F7B50400808801F0D3FF0025A84203D019
:106A20000578A08802F008F81C4E3378002B1FD0A0
:106A3000AB421DD11A4B28001978FFF777FF0028C9
:106A400018D000233370A3790820A778A688019373
:106A500005F0E6F8011E0DD0D0230370CA3B837009
:106A6000019B477086808371280005F001F801E0E2
:106A7000002DE8D1A0880B4B8200D358002B01D009
:106A8000FFF762FF1721A088FFF768FDA08801F0DB
:106A900027FDA08801F0FEFDF7BDC046A966FF1FD7
:106AA000A866FF1FB066FF1FF0B587B01D000CABD6
:106AB0001B88070001930DAB1B88142002930EABBB
:106AC0001B88160003930FAB1B880091049310AB37
:106AD0001B88059305F0A4F8041E1AD0D023037078
:106AE000CB3B47708370C670062229000430002D0E
:106AF00011D004F0FDFF019B21006381029B0098EF
:106B0000A381039BE381049B2382059BA37404F070
:106B1000AFFF07B0F0BD05F0F3F8ECE7F7B5009371
:106B200008AB1B8807000C200D001600019305F030
:106B300077F8041E13D0280001F042FF00280FD080
:106B40000078D0232370C93BA370009B21002381D0
:106B5000019B6770A580E680638104F089FFF7BD23
:106B6000014B1878EDE7C0460C45FF1F13B5040034
:106B700064890389C2888188C0780094FFF7CEFFBA
:106B800013BD000010B5044C2068002803D004F0A9
:106B900097FE0023236010BDB466FF1FA122F0B54D
:106BA000818892004A43384B384F1B6804009B1879
:106BB0009D2292009B18827989B01A603B68002B55
:106BC0005FD01D78324B1B68002B04D05B68002B14
:106BD00001D000209847260008363100E079FFF701
:106BE000B7FD237DE0710200E0780493638A2900F9
:106BF0000393238A0293E3890193A38800933300CC
:106C0000FFF752FFE378002B0BD1E289A379A1882B
:106C100002920196E27928000092012201F0DAFE48
:106C2000E0703B68002B20D0FFF7ACFF194D2878AF
:106C300000281AD0184B1978FFF778FE002814D0D6
:106C40002B78E67808200793A78804F0E9FF011E57
:106C500009D0D0230370CA3B467083708780867149
:106C6000079804F005FF00232B701721A088FFF779
:106C700075FCA08801F034FCA08801F00BFD09B080
:106C8000F0BD064B9DE7C0463409FF1FB466FF1FE9
:106C9000C866FF1FA966FF1FA866FF1F0C45FF1FE0
:106CA000F8B5070008000E0001F08AFE041E18D097
:106CB0002620FFF78DFC051E00D12578062004F064
:106CC000AFFF041E0DD00021062205F019F8D023D5
:106CD0002370C23B21006770A370A680E8B204F065
:106CE000C7FEF8BDF0B585B001930AAB1B7807006D
:106CF00002930BAB1B7808000D000092039301F088
:106D00005FFE061E22D0102004F08AFF041E1DD054
:106D10001022002104F0F4FF2620FFF759FC002880
:106D200000D13078D0232370C13BA370009B210099
:106D30002372019B67706372029BA580A372039B01
:106D4000C0B2E3720C9BE36004F092FE05B0F0BDAC
:106D5000F7B50D00019001F033FE071E20D00E2084
:106D600004F05EFF041E1BD02620FFF731FC061E38
:106D700000D13E78D0232380C53B0622A370F91DA5
:106D8000E01C04F0B5FE019B2A0063810123DD4075
:106D90001A401D40210022736573F0B204F068FEB2
:106DA000F7BD0000F0B585B0029010000D0017008F
:106DB0000A9E039301F004FE041E31D0029B002BB7
:106DC0002ED1039B02795B0724D51223134304229F
:106DD000002E08D10B99002905D10C99002902D168
:106DE0000D9900291AD01A430D9B2271002B00D057
:106DF000C9E0002E00D1CFE0002D00D0CCE0606AC9
:106E0000002801D004F05CFD1C21300004F0B8FD26
:106E1000606205E002239A430E33D7E79343237160
:106E2000654BBA00D458002C00D1AAE0002E10D037
:106E3000236A002B03D11C2004F082FD20625E4BEC
:106E4000BA00D358186A002803D01C22310004F07D
:106E50004FFE0C9B002B12D0574CBB001D596B6A88
:106E6000002B03D1162004F06BFD6862BB00E358D1
:106E7000586A002803D016220C9904F039FE0D9BA5
:106E8000002B11D04C4DBC006659B36A002B03D1C6
:106E9000142004F055FDB0622B59986A002803D0E5
:106EA00014220D9904F024FE380001F089FD051E1E
:106EB00067D0414BBA00D358002B62D01A6A3420F5
:106EC000002A00D11C389A6A002A01D0143080B2FE
:106ED0000B9A002A01D01C3080B25B6A002B01D0D3
:106EE000163080B204F09CFE041E4AD01822002105
:106EF00004F006FF2620FFF76BFB0190002801D16C
:106F00002B780193D0232370029B200063700A2307
:106F1000294EA370039BBD00A371AB59A780196ACA
:106F20001830002905D01C22A06004F0E1FD2000EB
:106F300034307359996A002907D00300142214339E
:106F4000E060029304F0D4FD02980B9B002B08D064
:106F500003001C221C330B992061029304F0C8FD2E
:106F600002987359596A002903D01622606104F00F
:106F7000BFFD6B462100187904F07AFD3800FFF759
:106F8000E3FC05B0F0BD10220D9B0D991B69A01804
:106F9000236204F0ADFD2CE70B9B002B00D13FE7F3
:106FA000012D00D03CE7606A002801D004F088FC85
:106FB0001C210B982AE7C046B066FF1F10B5044C91
:106FC0002068002803D004F07BFC0023236010BD60
:106FD000A466FF1F0B4B07B51A68002A01D10020D9
:106FE0000EBD6946531C012012780731FFF772FC71
:106FF0000028F4D002780123100018401A42EED085
:10700000EEE7C046C066FF1FF0B51F4F01203B688A
:1070100087B0002B25D09B78059300F0B3FB0028A8
:1070200021D00A20FFF7D4FA04000B20FFF7D0FA92
:10703000164B05001E78731E9E413B68F6B2191D63
:10704000D878FFF757FB3B682900DA7A04330392BC
:107050009A7901930292009033002000059A04F07F
:107060004FFB07B0F0BDFFF7B5FF002805D00620A5
:10707000FFF7AEFA04000720D8E70820FFF7A8FAC8
:1070800004000920D2E7C046A466FF1FA066FF1FC8
:1070900070B50A4E040033780D00FF2B0DD004208C
:1070A00004F0BEFD011E08D0D0230370CE3B457016
:1070B0008370C470307804F0DBFC70BD1C45FF1F8A
:1070C00070B5040006200D0004F0AAFD011E0AD0D0
:1070D000D0230370CD3B8370054B44701B688580C3
:1070E000187804F0C5FC002C01D0FFF767FF70BDD5
:1070F000A466FF1FF8B5264F06003B680D0011245B
:10710000002B05D10522234B1B78134202D11224F8
:107110002000F8BD204A10241268002AF8D0127806
:10712000002AF5D0DB0719D52B789A1E012A1AD828
:107130000C2004F005FC132438600028E8D000235C
:107140000A22437029000670023004F0D1FCFFF7D8
:107150005BFF041E0AD0FFF731FFD9E700F012FBF6
:107160000028E1D1E4E7002BE2D0D0E70B4B1B78FD
:10717000032BCDD11D20FFF72BFA094B18800028D7
:10718000C6D0084B04211878074A04F009FDBFE770
:10719000A466FF1FA166FF1FC066FF1FA066FF1F3A
:1071A0009E66FF1FCC66FF1F60EA0000F7B50193E3
:1071B000194B14001A78052306000F0012201A42FA
:1071C00021D0012920D1154B1D68002D1BD0022094
:1071D0001F2C18D8002C02D0019B002B13D0104B71
:1071E0001F221E706E1C0021300004F089FD0199E1
:1071F0002200300004F07CFC310020002C70002FB5
:1072000006D004F08DFCFEBD064B12201D68DCE7A5
:1072100004F00EFBF7E7C046A166FF1FC066FF1F24
:107220001C45FF1FBC66FF1FF8B50F4E12243368C4
:10723000002B17D01B780F3C834213D100250B4F36
:107240000221387804F0B4FC094B042138781D8001
:1072500004F0AEFC074B28001D8033685C7004F01E
:107260001FFD04002000F8BDA466FF1FCC66FF1FB1
:10727000B866FF1F9E66FF1F70B5012823D11B4C07
:107280002388002B03D01A4A1578002D07D0194BFC
:107290001B68002B02D01878FFF7C6FF70BD3B2B90
:1072A00002D93C3B2380F9E7134E0221307804F0E9
:1072B0007FFCFA222388920002215A43307804F09E
:1072C000F7FA2580EAE70B4B1B68002BE6D00B4B47
:1072D0001B785B07E2D5084B0221187804F068FCA4
:1072E0000022024B1A80FFF769FED7E7B866FF1F3E
:1072F0009C66FF1FA466FF1FCC66FF1FA166FF1FD1
:10730000F8B51E4D2868002803D004F0D9FA0023F0
:107310002B601B4E3068002803D004F0D1FA002304
:107320003360184F05243B7818002040234221D0B9
:10733000154800F02BFA3B78234213D0202004F0AC
:10734000FFFA2860002813D02022002104F0D8FC86
:10735000202004F0F5FA041E306005D02022002120
:1073600004F0CEFC002004E0286804F0A9FA2C60A8
:107370001320F8BD00F00AFAF4E7C046C066FF1F0C
:10738000BC66FF1FA166FF1F1045FF1F10B50A4C0A
:1073900023681A1E0ED0002808D10130587004F05E
:1073A0007FFC002805D02368002B02D00021FFF7C6
:1073B00087FE0122100010BDA466FF1FF7B5274EFF
:1073C000050033680191181E21D05C78244F012CF0
:1073D00030D1FFF7FFFD002825D02000FFF7F8F897
:1073E0000400412814D91F4B022118781E4A04F0CA
:1073F000D7FB1E4B3C3C1C80022233685A703B7802
:10740000002B14D128000199FFF75AFE0120FEBD80
:10741000FA2292004243002AEED0124B0221187841
:1074200004F046FAE8E7FFF7D3F80200F3E7002399
:107430003B70EBE73B78002BE8D1032004F0F0FB36
:10744000011E08D0D0230370CC3B45708370336895
:10745000187804F00DFBFFF7B1FDD7E7A466FF1F16
:107460009C66FF1FCC66FF1F60EA0000B866FF1F26
:1074700010B51749838802008B4220D011D81549D6
:107480008B4217D0144900205B1899B2012907D804
:10749000926811785A425341D8B2FFF7F9FD0120A2
:1074A00010BD0E4A00209B1807229BB29A42404111
:1074B000C0B2F5E783681878FFF768FFF0E78368E4
:1074C00099785A78090218781143FFF777FFE7E7B0
:1074D0000A20000006200000F8DFFFFFAFDFFFFFFB
:1074E000014B18707047C0461D45FF1F10B5064C74
:1074F000207001F041FA207804F01AF90521207873
:1075000000F062FD10BDC046CC66FF1F0BB273B524
:107510000D00002B00DBC4E0884B187804F098FBCA
:10752000041E0ED00378912B0FD0A22B00D1A1E026
:10753000834B1878FF2852D0210004F099FA0028D4
:107540004DD180200002684076BD43780F2B76D065
:1075500013D8052B70D00E2BEAD18088794B984236
:107560002BD8794B98421BD8784B9842E0D1A3682E
:107570001878591CFFF774F838E03E2BD8D183787F
:10758000032B74D06CD8012B6ED0022BD0D1704B52
:107590001B68002B23D05B68002B20D098471EE08F
:1075A0006C4BC0180C28C3D804F072FA1DC2C21567
:1075B0000BC20B0B0B3223C23C00674BC0180728D1
:1075C000B6D8664B1B68002B09D01B68002B06D071
:1075D000200098470AE0A3681878FFF7C7F8200052
:1075E00004F0C6FAADE7A068FFF762F800289FD064
:1075F000F5E7A3681B78002BF1D0554B1B68002BD7
:10760000EDD01B68002BEAD0210055489847EDE7E4
:107610004F4B1B68002BE2D01B68002BDFD02100F2
:107620005048F3E7504B1B68002BD8D05B68002B09
:10763000D5D021004348E9E7FFF7EAF9CFE7808892
:107640004A4B984203D04A4B984200D070E7464BD1
:107650001B68002BC3D05B68002BC0D02100D5E78E
:10766000153B012BBBD963E7FFF798FAB7E7FFF7A4
:107670007DFAB4E73F4B1B78042B07D100236A4601
:1076800013800179408800F0C5FCA8E7364B1B68E1
:10769000002BA4D05B68002BA1D00100364898478E
:1076A0009DE7012421420AD0294B1B68002B04D0FE
:1076B0005B68002B01D000209847012043E78B072F
:1076C0000AD5264B1B68002B04D05B68002B01D029
:1076D00020009847022036E70421280008400D4288
:1076E00000D131E7254E3388002B21D0013B9BB2DE
:1076F0003380002B1AD1FFF7DBF800280AD0204B8B
:107700001C70164B1B68002B04D05B68002B01D04B
:1077100020009847FFF7C6F8694601F001FD68466A
:10772000FEF7FEFF1D20FEF753FF308004200AE71E
:10773000024B187804F03CFAF8E7C046CC66FF1F0D
:107740001D45FF1F0E200000012000000910000051
:10775000C466FF1FFEDFFFFFAFDFFFFFC866FF1F2E
:107760000C2000000B200000AC66FF1F0D20000065
:1077700013200000A166FF1FFFFF00009E66FF1F91
:107780009C66FF1F10B501F09BF910BD014B1860FE
:107790007047C046C866FF1F0B880020162B01D813
:1077A00017230420014A13807047C0467666FF1FE6
:1077B00000207047074A03001188814207D0918852
:1077C0000020994202D1013080001018704700203B
:1077D000FAE7C046D466FF1FF0B58F7806000D00AB
:1077E000C7B01E2F15D1FFF7E5FF051E03D10024FA
:1077F000200047B0F0BD00223B003100C07800926D
:1078000000F0B2FB0400A81C00F0D3FBFF23EB70D8
:10781000EEE7264B062403931B78FF2BE8D0182FA6
:10782000E6D87B08224A013BDB0002929A58944634
:10783000002ADDD0029AD3185B68002BD8D00878D4
:10784000002802D14B78012B02D10624122FCFD170
:1078500007AFAB88697800976446AA68A047041E02
:10786000C6D1AB78029A5B08013BDB00D318390024
:1078700030005B689847041E0BD1AB78042BB6D060
:10788000039A310010782200009700F06DFB04008D
:10789000AEE76A78002AABD1AA7805A93B880871BF
:1078A00030000A704B80FEF747FBA0E72045FF1F22
:1078B0003CBF00111D4B37B5050098420BD0002985
:1078C0000AD1FFF777FF002805D11948FFF772FFAB
:1078D000002800D0058037BD01291AD1FFF76AFFC3
:1078E000041EF8D001235B420380A378FF2BF2D063
:1078F000FE2B07D00023E0781422009329001E33CA
:1079000000F032FBA01C00F054FB01235B426380BB
:10791000E1E70229DFD1013901F0BEF80028DAD110
:107920002800FFF747FF041EDFD1D4E7FEFF000069
:10793000FFFF0000022210B5074B52421A80074891
:1079400001325A809A80DA8000F07EFA044801F011
:1079500025F8002010BDC046D466FF1FD97700115E
:10796000B57800110388F7B50400002B02D1022579
:107970002800FEBD42680221137825485268FEF7B0
:10798000A5FD00282ED0234F01253A88002AEFD0EC
:10799000802321885B0201259B1A9942E8DC0C2098
:1079A00003F0CEFF061E31D03B8822889C46002380
:1079B0001800019561469DB2491989B2AA421BD8A7
:1079C000002801D062443A8000233000082208C019
:1079D000210004F08DF8104A1368002B13D1002504
:1079E0001660C5E76268022113780C485268FEF7FA
:1079F0006DFD0028C7D1BAE760681D0140194181BB
:107A000001330198D6E71A001B68E6E71325AFE7B4
:107A1000AABF00111E45FF1FD066FF1FA8BF00119F
:107A2000014B18707047C0462045FF1F14230A0001
:107A300010B51A40194204D00122102101F048F873
:107A400010BD4B06F9D4012088434000F8E710B57B
:107A500014008B0604D50122102101F039F810BD65
:107A600008230A001A40194202D14BB2002B0FDA48
:107A7000102101F02DF8002808D02300F9331B78DD
:107A8000002BECD0F8342378012BE8D10020E6E776
:107A900003208907FAD4E2E7F0B51F00184B85B040
:107AA0001C68019002910392002C27D1200005B0A0
:107AB000F0BDA5683301ED186B89019A934211D38B
:107AC000029A93420ED8002F04D10A9B002B10D1AA
:107AD0002C00EBE73B002978039A6868FEF7F6FC78
:107AE0000028F2D10136B6B2A388B342E1D82468A7
:107AF000DAE7A3680A9A5B891380E9E70026F3E7CF
:107B0000D066FF1F37B50C000A88498801239142CF
:107B100017D3002A15D0651D23792A0002210A48AF
:107B2000FEF7D4FC102300280BD02379618820882D
:107B300000242A000094FFF7AFFF0A23A04200D0E0
:107B4000230018003EBDC046AABF001113B50A00AD
:107B500008884988012388420BD8002809D00024CE
:107B6000137905320094FFF797FF0A23A04200D053
:107B70002300180016BD13B50A00088849880123A0
:107B800088420BD8002809D00024137905320094CC
:107B9000FFF782FF0A23A04200D02300180016BD81
:107BA000F0B58BB003904A8808880E00012382420A
:107BB00055D3002853D00023012704AC23700022A2
:107BC000718813000092FFF767FF051E3ED02078F2
:107BD000002835D12B78022B18D167706A89830071
:107BE0000130E31880005A8069680222201803F0EF
:107BF0007FFF23780133DBB22370042B19D93B00BC
:107C00006889013080B2002BD9D01FE00223637055
:107C1000122358436A89231804305A806968102255
:107C2000201803F065FF23780133DBB22370002BAB
:107C3000E5D10C4A6B899B185A425341DBB2DFE70E
:107C40006378012BE4D12B78022BC7D022780A234A
:107C5000002A04D021000398FEF798F900231800A9
:107C60000BB0F0BD0100FFFF0F4BF0B5040018682A
:107C7000002816D083685D89A54207D88288AE188F
:107C8000B44203DA12019A18934201D10068EFE777
:107C90001E005F891036A74204D1002900D00D8054
:107CA0001800F0BD3300EFE7D066FF1F70B5050088
:107CB0000C0008880021FFF7D7FF03000120002BEC
:107CC00004D022002800197AFFF7C1FE70BDF7B575
:107CD0000C00002501902300F6331B78AB4201D83D
:107CE00000200AE06B00E65A00213000E718FFF799
:107CF000BBFF002802D126800130FEBD017A019829
:107D0000FFF794FE002802D03B882380F5E7013579
:107D1000EDB2E0E710B5040008880021FFF7A4FFEA
:107D200003000120002B03D02000197AFFF77EFE0C
:107D300010BD0000054B1B68002B01D1180004E0AA
:107D40009A6852898242F6D198887047D066FF1FA0
:107D5000F0B50E27002687B0039302ABFF183E80D4
:107D600005001F4B40891400984207D02B78013042
:107D700000976A6880B2FFF78FFE060002212B7819
:107D800018486A68FEF7A2FB00280FD06C89200013
:107D9000FFF7D0FF002802D0013C0419A4B2039BD6
:107DA000002B00D01C80300007B0F0BD02212B78E2
:107DB0000D486A68FEF78AFB0028E7D102212B787C
:107DC0000A486A68FEF782FB002807D0002EDED042
:107DD0003B88A342DBD17489013CDFE76C89DEE795
:107DE000FFFF0000AABF0011A8BF0011A6BF00112D
:107DF00010B50C00FFF7DEFC03000220002B0AD0B8
:107E0000002C00D023609B781720FE2B03D0013874
:107E1000FF2B00D1002010BD73B50D0001A9040097
:107E20001600FFF7E5FF172805D0002E04D1290022
:107E30002000FEF727F976BD01221021200000F076
:107E400047FE0028F3D0F6E7014B18607047C046A4
:107E5000E066FF1F37B56B469D1D0100040002223E
:107E6000280003F0BDFC2B88B02B0ED12379122BF8
:107E700009D12300FF339B78012B06D101216088B3
:107E800000F0E0F801E01B2BF8D037BD10B5054B32
:107E90000421187000F098F8FFF74CFDFEF770FB16
:107EA00010BDC046E466FF1F0020F0B50BB20F0006
:107EB00087B0834234DA274B187803F0C9FE051ED9
:107EC0002BD00378A02B25D103AE3100FEF7E4F8C8
:107ED000041E0BD1B378DB0724D51F4B06341B6877
:107EE000002B03D03100688898470400A868002858
:107EF00001D003F0A5FC002C08D1184A039B1340C5
:107F0000174A934206D0B3781B2B03D0012168880F
:107F100000F098F8280003F02BFE80200002784043
:107F200007B0F0BD0F4B1B68002B10D031006888E4
:107F30009847041EDAD07378002BD7D1B27801A904
:107F40000A704B800C716888FDF7F6FFCEE70624B7
:107F5000F1E7C046E466FF1FDC66FF1F00FFFF007D
:107F600000011200E066FF1FF7B50190822040007B
:107F70000D0017001E0003F053FE04001320002C18
:107F800012D0B02320002370089BFC22677065800C
:107F900026710830002B08D0190003F0A9FD21003C
:107FA000019803F065FD0020FEBD089903F0A8FECE
:107FB000F5E710B5041E06D00078FD2803D803F0BD
:107FC000FFFCFF23237010BD0A1F93B210B50400FD
:107FD0000220032B05D882400020024BD1529B186F
:107FE0009C7010BD0467FF1F0B8870B5043B040034
:107FF0000D000220032B0BD80121200000F04CFDC6
:1080000003001420002B03D02900200000F0DEFB29
:1080100070BD000007B51300034A00920A00012159
:1080200000F02CFC0EBDC0465182001107B5019234
:1080300003220092024B0A00122100F049FC0EBDFF
:10804000CF82001107B56B4601AA11800449D88080
:1080500008780633012802D1190003F099FC07BD06
:10806000E566FF1F0C4B10B518700023FF210B4A6B
:108070001380138193819380094A53801370517246
:1080800093819372D174D3821375517703F060FD9D
:1080900000F0FCF910BDC0461467FF1F0467FF1F06
:1080A000E666FF1FF0B58DB06B46002003910C22F1
:1080B0009B5E834200DBB0E05D4B187803F0C8FDA7
:1080C000051E00D1A4E00378902B00D09DE006AF00
:1080D00001004688380000F013FA7968040000298E
:1080E00000D19CE03B88052B6ED13B89032B1CD92A
:1080F00005AC200000F0A2F86288172A61D83989FF
:10810000131D994231D17968237804310291D9073E
:1081100038D5607800F08EF9071E06D00023037171
:108120002378012B08D0132B23D0A868002800D176
:1081300078E003F085FB75E06288029909A800F0F9
:10814000A6F80290380000F08BF909AA2378387A53
:108150000192002231000092029A00F012F93800D8
:1081600000F064F9029B002BDFD0300000F080F9B2
:10817000DBE70378032BD8D16288029909A800F0C5
:10818000D6F8DEE7122B13D1029909A800F0B5F852
:10819000021EEAD127498B88002BC6D0887909A90D
:1081A0002378019161780091310000F0EAF8BCE792
:1081B000002302AA93833000617809AAFFF72AFFFF
:1081C000B3E71D4B0993F6E7042B02D09A1F012A4F
:1081D000ABD8184A043B9B00995A0029A5D0D21865
:1081E000907831003A0000F0AEF800289DD13B882D
:1081F000042B03D001213000FFF724FF012C04D110
:10820000A868002801D003F01BFB280003F0B0FC95
:108210008020039B0002434018000DB0F0BD0128F0
:1082200000D182E701213000FFF70CFFEDE7C046E7
:108230001467FF1F0467FF1F010017000B7803700E
:108240004B784370CB788A781B0213434380704786
:108250000A88030002700A88120A42700A88012AFA
:1082600006D14A8882704A88120AC2700420704778
:1082700002208242FBD14A8804309A704A88120A4E
:10828000DA708A881A718A88120A5A71EFE710B573
:108290000400012082420CD94B780A781B02134358
:1082A0002380834206D1CB788A781B0213436380F4
:1082B000002010BD022BFBD1CB788A781B02134320
:1082C00063804B790A791B021343A380F0E70B8884
:1082D00003700B881B0A43704B8883704B881B0A02
:1082E000C3708B8803718B881B0A4371CB888371A1
:1082F000CB881B0AC3710820704703000120082A9D
:1083000014D14A780878120202431A80CA78887811
:10831000120202435A804A790879120202439A8073
:10832000CA798879120202430020DA80704710B5BA
:1083300004000120022A05D100204B780A781B0294
:108340001343238010BDF8B5060010200F00150060
:1083500003F066FC04000120002C0ED0A0230C22A8
:10836000290023806780201D002D07D003F0C0FB6B
:108370002100300003F07CFB0020F8BD03F0C0FCBE
:10838000F6E7F7B51E00009008AB142017001D7823
:10839000019103F045FC041E12D0A2230370019B3F
:1083A00047704380099B057146710C220830002BF1
:1083B00007D0190003F09CFB2100009803F058FB44
:1083C000F7BD099903F09CFCF6E737B5041E0FD002
:1083D0004388002B0CD00025C1881323007A172274
:1083E00001950095FFF7CDFFFF236580637225702F
:1083F00037BD000010B50C4904004A88002A09D096
:108400008B89002B05D00020CB8A0222834201D029
:1084100010BD012213000A20434300204032C854FB
:10842000C81842800472F3E7E666FF1F002343800A
:1084300003707047094B00211A0010B55C88002CAE
:1084400006D01C79844203D10A234B43D01810BDB7
:1084500001310A330329F1D10020F8E7E666FF1F56
:1084600010B50400407A03F0ABFAFF23637210BD2D
:108470007047043010B580B203F052FA002803D0E0
:108480000421494203F094FA10BD000070B50025A4
:10849000104CA0682580A581A580A84202D003F0D9
:1084A000CFF9A56000250C4C0C4B606D1D8023009E
:1084B00058331D70A84202D003F0C2F9656500254B
:1084C0006068002801D003F0BBF9013508340A2D9B
:1084D000F6D170BDAC67FF1F5067FF1FA067FF1F7D
:1084E00070B5041E09D1054D2880A881A880A86810
:1084F000002802D003F0A4F9AC6070BDAC67FF1F88
:10850000F0B54B8885B00193002343600A790500DC
:108510000F00022A00D07BE0CA88032A17D98B6893
:108520005E7819783602DC78D8790E4399781B7A10
:1085300024021B020C43034353495BBA0B80331DD7
:1085400093421ED1042C04D0631F022B0ED90120AC
:1085500015E0019A4D4B1201D35A002B06D0019819
:10856000FFF7BEFF4A4A1369013313610421B8685B
:108570002E812C80494203F01BFA6860002005B070
:10858000F0BD434D042C06D0631F022B0FD9EB68BE
:108590000133EB60DBE7019A3C4B1201D35A002B0D
:1085A00005D00198FFF79CFF2B6901332B61374BF6
:1085B00030000293019B029A1B0101930023019951
:1085C0008C468B52130063449C8003939E81FFF77B
:1085D00050FF039B041E986016D00421B8684942DE
:1085E00003F0E6F9FA880100043A200003F080FA6B
:1085F0000199029AFB888A5A043B9B18029A8B5273
:108600002B6801332B60A2E7AB690133AB619EE7B6
:108610001E4B0293019B1E01029BF35A002B2DD08F
:1086200002998C19A068002828D0012A26D1FA883E
:108630009B189BB27352A189994217D39B1AC018F9
:10864000B96803F055FA029BA289F35A934200D00D
:108650007DE700222B81A3882B80A3686B60029B9F
:10866000F2520B4A53680133536070E7084A93682B
:10867000013393600198FFF733FF68E7044A5369B9
:1086800001335361F6E7C0461667FF1FAC67FF1F53
:108690001C67FF1F70B5051E15D10B4C0B4B1880C6
:1086A000230058331870606D002802D003F0C8F81A
:1086B0006565250050356068002801D003F0C0F8DA
:1086C0000834AC42F7D170BD5067FF1FA067FF1F91
:1086D000F0B51700A12285B0920001934243394BB7
:1086E00006001B680C009B18D933FF331D78FDF77B
:1086F00041FF0430854204DD3000FDF73BFF0430CC
:10870000C5B2BD4207D33A0000213000019B03F0FF
:1087100027FA05B0F0BD2900380002F0E9FF230078
:10872000C6B250331E700393019B29006365380065
:1087300003F0AEFACBB20293002B02D0039B0136BA
:108740001E7000262300503303931B78B34204D8D5
:10875000606D002831D10020DBE7029A2800002A52
:1087600004D0013B1000B34200D02800F700E71905
:10877000387002F0EDFF786000280ED03A78019949
:1087800003F0B6F9019A3B780136D3180E4A0193EB
:10879000D369F6B20133D361D4E7039B18706065E7
:1087A000A74205D1084A1320D36A0133D362B0E748
:1087B000606803F045F80834F2E703F041F800235D
:1087C0006365C8E73409FF1F1C67FF1FF7B50D007D
:1087D00007000421686803F0EBF82B89040003709C
:1087E0002B891B0A43702B8883702B881B0AC3704C
:1087F0002E8902250436F6B2FB2E15D81B4B9F425C
:1088000014D10C2003F00CFA1135011E0CD090236A
:1088100003708E3B0371043B4380154B8460C6801C
:10882000187803F025F900252800FEBD5C237B4362
:10883000104AD3180093583301931B78002B0FD1A3
:108840000300320038000099FFF742FF019B05004A
:108850001B78002BE8D13800009903F0A1F8E3E77A
:10886000054A0725536A01335362DDE7FEFF000026
:108870001467FF1F5067FF1F1C67FF1FF0B587B00D
:10888000009017200F0016000193FFF7F2FD13254B
:10889000041E19D00C98031E02D00199201D984780
:1088A000030AE370052302AAA070043090812770A8
:1088B0000098667003A993800494FFF787FF051E54
:1088C00002D0200002F0BCFF280007B0F0BD00007D
:1088D000F0B587B01F000CAB1B7803910593012105
:1088E0000DAB06001C78049200F0D6F81425002881
:1088F00021D02000FFF77EFD0135041E1BD0114959
:10890000059B0A7803700132D2B2131EC68001D1D2
:1089100001231A000B7022713000049B0399009709
:10892000FFF7ACFF051E09D1230021000648074AC6
:10893000093302F0ADFF280007B0F0BD00236380CB
:108940002370F8E71867FF1FCB8300113075000014
:10895000F8B505000E00064C064F2368002B02D028
:108960003100280098470434BC42F6D1F8BDC04617
:10897000BC67FF1FD067FF1F0123064A5B4253807D
:10898000002313715362044A136053609360D360F1
:1089900013617047D067FF1FBC67FF1F02000023F1
:1089A00010B506499C000859002801D1625010BD3D
:1089B0000133052BF6D11320F9E7C046BC67FF1F32
:1089C000034A5388181A43425841404210407047A6
:1089D000D067FF1FF0B585B002930AAB1F780CABD0
:1089E0001B88009008000E0001920393FFF7E8FF38
:1089F00005001120002D1BD10E48FFF7E1FF0400F8
:108A00001520002C14D006220B99A771E01D03F04D
:108A10006FF8019B30002371029B29006371009B5A
:108A200066802370039B6562E381FFF791FF280056
:108A300005B0F0BDFFFF000010B5FFF7C1FF040057
:108A40000220002C12D060880121FFF781FF606AAC
:108A5000002801D002F034FF28220021200003F07A
:108A60004FF9012300205B426380207110BD00009C
:108A700030B5074A074C5588010013780020A542FD
:108A800004D05B1A59424B415842104030BDC04699
:108A9000D067FF1FFFFF0000084A10B501230C003C
:108AA000904208D0FFF78CFF031E04D003792340C7
:108AB0005A1E9341DBB2180010BDC046FEFF0000F5
:108AC000024B1879431E9841C0B27047D067FF1F10
:108AD00070B504000D001600FFF772FF002804D1E6
:108AE0000D4B9C4200D0143070BD416A03790520C3
:108AF000002907D012221A40102A02D10520002E88
:108B0000F2D10F20DB06EFD5897E0C20A9428941E6
:108B1000494249420840E7E7FEFF0000030010B564
:108B2000002800D110BD0348034A41889142F9D082
:108B30009847F7E7D067FF1FFFFF0000002330B51D
:108B4000C45CCD5C6C40D4540133102BF8D130BDE3
:108B50000F23002210B5C45C64002243CA54C25CD7
:108B6000D209013BF7D210BD0200010010B520323E
:108B7000103102F00DFE10BDF0B58BB00390102047
:108B800005931700049102F0DBFE0090102002F024
:108B9000D7FE009B13240190002B05D000280CD198
:108BA0001324009802F08CFE019B002B02D01800C9
:108BB00002F086FE20000BB0F0BD102002F0C0FED7
:108BC0000600102002F0BCFE13240500002E00D188
:108BD000AEE0002819D01022002103F091F83200F5
:108BE0002900039802F0D4FD041E0ED133787F2BA8
:108BF00051D830000099FFF7ABFF009B1B787F2B0B
:108C000053D801990098FFF7A3FF300002F058FEF7
:108C1000002D02D0280002F053FE002CC1D11020FC
:108C200002F08EFE0600102002F08AFE0290002E56
:108C30007CD0002878D03A000F3223000125121191
:108C400005D00F333B4015B25A4253411BB26A1E46
:108C50001201002B33D0049BD2B298180099029ACB
:108C6000FFF76CFF013D10220021300003F048F8AF
:108C7000ADB2049F2D017D19AF4242D0002C33D0FC
:108C8000300002F01DFE029B002B00D189E7180086
:108C900002F016FE85E729003000FFF759FF280093
:108CA0002549009AFFF74AFFA7E729000098FFF738
:108CB0004FFF28002049019AFFF740FFA5E70F2149
:108CC0000F4004998A18D9B28F4208D9D15C06A8FE
:108CD00019540133102BF6D1029A0199C0E7791A81
:108CE00048424141C901F2E73900300006AAFFF7C6
:108CF00025FF3200039806A902F04AFD1037040050
:108D0000BAE7002CBCD13000029906AAFFF716FF83
:108D1000320006A9039802F03BFD0822040031004E
:108D2000059802F0E5FEABE71324A9E71324AAE7B0
:108D3000002800D06EE733E7B0BF0011F0B58BB06C
:108D40000F0016000225009000283FD0002A3DD0D9
:108D50000B1DDBB21800029302F0F2FD1135041E68
:108D600034D0FDF747FD05003A000099201D02F0C0
:108D700077FEEBB20393E3702B0CDBB22F0A009368
:108D80006370FFB22B0E2370A7700193FDF72CFDCB
:108D90001022010006A802F063FE2100029A04AB33
:108DA00006A8FFF7E9FE051E0DD1039B08223370CC
:108DB000009B04A9B370019B7770F370301D02F023
:108DC0004FFEFDF71DFD200002F07AFD28000BB0DC
:108DD000F0BDF0B58FB00D00149E03900492059382
:108DE000002A03D1022420000FB0F0BD002EF9D0DC
:108DF0000398FFF7E5FD1424071EF4D0727833784A
:108E000012021A43B3781B041343F27812061A4372
:108E1000036A0192934201D30133E3D1002D03D0C1
:108E20003B7901249B07DED50822002106A802F029
:108E300067FF059B13240433DBB21800029302F092
:108E40007FFD051ECFD0059A0499043002F008FE7C
:108E500004223100280002F003FE390010221031F4
:108E60000AA802F0FDFD2900029A06AB0AA8FFF746
:108E700083FE041E0FD1082206A908A802F0F0FD07
:108E80000822311D08A802F0C3FC012807D101996E
:108E90000398FDF7C9FC280002F012FDA3E70124A6
:108EA000F9E7000070B51C4C05002368181E10D0AF
:108EB000002D14D11A78002A0CD1981C083202F027
:108EC00017FE02F015FD0135002808D123681D703A
:108ED000012070BD0A331800082202F009FE236841
:108EE000002BF5D0122002F09BFE061E0DD0C123F0
:108EF00021680370457002311022023002F0F8FD43
:108F000023683100587802F0B3FD206802F0D8FCE5
:108F100000232360DCE7C046F867FF1FF8B50400B4
:108F20002020FDF755FB0D4EA700BB590500002B77
:108F30000DD000280BD0D878FF2809D108492A0085
:108F40000C55F35907480333611802F0A1FCF8BD32
:108F5000290002F095FD0028F0D1F8E71468FF1F02
:108F6000FC67FF1F75A1001170B5064D84006359A1
:108F7000002B05D0D87802F023FDFF226359DA7068
:108F800070BDC0461468FF1F70B506008CB00C00A1
:108F9000150000213022684602F0B2FE3100102296
:108FA000684602F05DFD1D2021000322684402F0A6
:108FB00057FD6846FFF7D8FD2D2104000322280045
:108FC000694402F04DFD20000CB070BDF0B5070003
:108FD000160097B001931CAB1D7830221EAB009198
:108FE0000AA800211C7802F08BFE102239000AA882
:108FF00002F036FD1022002102A802F081FE0722B5
:10900000310002A802F02CFD072202AB9818631E63
:109010009C41019902F024FD02AB9C732B005A1E67
:10902000934102AAD3730021102206A802F068FE21
:1090300006221D9907A802F013FD1A2002ABC018E2
:1090400006221F9902F00CFD102200990EA802F0D2
:1090500007FD102202AB0EA908781C78013A604087
:10906000D2B2087001330131002AF5D10AA8FFF706
:109070007BFD102212A904000EA802F039FD102277
:1090800006AB0EA908781D78013A6840D2B2087084
:1090900001330131002AF5D10AA8FFF765FD044329
:1090A00010222098E4B212A902F0DAFC200017B0D6
:1090B000F0BD70B50E0014008CB00100102268469F
:1090C0001D0002F0CDFC3100082204A802F0C8FC0B
:1090D0002100082206A802F0C3FC6846FFF744FD01
:1090E00004001022280008A902F0BAFC20000CB0ED
:1090F00070BDF8B506000D0000243719AC4200D34E
:10910000F8BD02F06DFC030A3B70631CDBB2013753
:109110009D4203D90234F054E4B2EEE71C00EDE7BF
:1091200073B506000C000225002819D0002917D0BD
:10913000032101A8FFF7DDFF6B469A793F231A4010
:10914000013313436A463000937101A92200FFF7EF
:109150001BFF051E04D10322E01C01A902F0C8FC7C
:10916000280076BD03785807DA08C00FD2008000C7
:109170009B0710439B0F1843C0B2704707230B4057
:10918000C908C9000B4303707047000070B50400A4
:10919000FFF7EAFE134DA4006359002B21D0186A93
:1091A000002801D002F08CFB2B59986E002801D0CA
:1091B00002F086FB2B59D86E002801D002F080FB0C
:1091C0002B59186F002801D002F07AFB2B59586FE9
:1091D000002801D002F074FB285902F071FB002333
:1091E0002B5170BD1468FF1F0E4B8000C35870B523
:1091F0000C00002B0FD09D68002D0CD02B78201D6B
:109200000B706B784B70A97CFFF7B8FF2B7E237235
:109210006B69E36070BD10220021200002F070FD38
:10922000F8E7C0461468FF1F014B18607047C0463E
:109230001068FF1F074A03008000825810B5002AFB
:1092400006D0D088984203D1012901D1FFF79EFFB3
:1092500010BDC0461468FF1FF0B5264E95B08700BC
:109260000B93BB590500099112200A92002B31D0B3
:10927000D888FFF7A5FB04001420002C2AD0280072
:1092800010A9FFF7B1FFBB591E781D6A002E23D02D
:109290000895FDF7EFFA07000020FDF7F1FA0790B7
:1092A000A379E61D069310AD0CA9089800F0E2FA28
:1092B0000EA9280000F0D7FA0B9B0A990493069B8D
:1092C00009980293079B0396019300970EAB0CAA93
:1092D000FFF77CFE15B0F0BDFDF7CCFA069030002C
:1092E000FDF7CEFAE31DA779079310AB06000893AC
:1092F000DAE7C0461468FF1F30B50C4C85002A59C8
:10930000030085B00120002A0ED018006946FFF73F
:109310006BFF2B591A78D888054B002A00D1054BD2
:109320006A46072100F0D9FB05B030BD1468FF1F65
:10933000679800117598001130B5094C85002959BE
:1093400085B010226846253102F0D2FB2A5911213E
:10935000044BD0886A4600F0C0FB05B030BDC04663
:109360001468FF1F1199001130B5094C8500295967
:1093700085B010226846353102F0BAFB2A59112116
:10938000044BD0886A4600F0A8FB05B030BDC0464B
:109390001468FF1F4F990011F7B54D4F860010203C
:1093A000F4590D0002F0CCFAF3592062186A132226
:1093B00000286CD0033A29009C6802F099FBF3590D
:1093C0001A780192002A58D11E6A227D317B944678
:1093D00051400122019F114201D167461740217D72
:1093E000914339432175377B4F40BC466046002787
:1093F000800701D44F081740012102208F40227DB1
:1094000082433A432275377B5740BC46604600276B
:10941000400701D497080F400420227DBF008243FB
:109420003A432275627D002794466046727B424033
:109430000A4201D167460F400121627D8A433A43C7
:109440006275777B5740BC4660460027800701D491
:1094500057080F400220627D7F00824317436775E3
:10946000767B00227E40760701D4BA080A400426A3
:10947000617D9200B1430A4362756A78002A08D080
:109480006278002A05D005220533DA770022100021
:10949000FEBD04222979114205D1A17C114202D1DD
:1094A0000533033AF1E7019A21782C78002A02D19A
:1094B0000A002100140018220429E8D8042CE6D858
:1094C00005206043034A05331218525CDDE7C046AD
:1094D0001468FF1FC0BF001110B50A001121024B14
:1094E00000F0FBFA10BDC046AB9900110B0030B57F
:1094F00087B001AD2B806B4604001100981D082237
:1095000002F0F6FA2A000B212000024B00F0E5FAE7
:1095100007B030BDD399001110B50A001121024BDC
:1095200000F0DBFA10BDC046279A001113B50B00FE
:1095300011006A4613706B4604000622581C02F0A4
:10954000D7FA6A4608212000014B00F0C6FA13BD85
:10955000479A001110B50A001121024B00F0BDFA24
:1095600010BDC046979A00117FB505000B4BAA00AD
:10957000D4580800002C0FD0666F237FE288217832
:109580000396266F0296E66E0196A46E0094FDF790
:1095900009FC2800FFF7FAFD7FBDC0461468FF1FD5
:1095A00010B51721FFF7E0FF10BD000070B50A00ED
:1095B0000D00064B0221040000F08FFA0600297806
:1095C0002000FFF7D1FF300070BDC0467799001131
:1095D00070B586B000236A461370836804001D7856
:1095E000681E0A2859D801A902F022FB0606333763
:1095F0003B3F43474B4F5300180000F042F906230E
:1096000012284BD000281BD16088FFF7D9F9082316
:10961000002813D04279002A47D1264B1A78072315
:1096200012070BD5244B1A680723002A06D01668A8
:10963000002E03D0290001AAB04703006A46137028
:109640006B461B786088002B2AD1FFF767FC06B0B9
:1096500070BD180000F06CF9D4E7180000F087F92D
:10966000D0E7180000F093F9CCE7180000F0ADF94E
:10967000C8E7180000F0C3F9C4E7180000F0F6F9D5
:10968000C0E7180000F0F6F9BCE7180000F013FA84
:10969000B8E7180000F013FAB4E707236A4613701E
:1096A00069466088FFF782FFD1E70523012AC5D10B
:1096B000024BB8E7A166FF1F0C68FF1F1068FF1F71
:1096C000F8B52C4F8600F35904000D00002B40D054
:1096D000DA8882423DD15A78062A33D11A78002A94
:1096E0002ED0012099681A6A097D014206D0157BA7
:1096F000054203D007225A700120F8BD0220014222
:1097000004D0157B054201D00922F4E70420014270
:1097100004D0127B024201D00B22ECE7164B1B68EF
:10972000002BE9D05B68002BE6D020009847BB599E
:1097300000215B78122BDFD12000FFF715FFDBE75C
:109740000E4BECE7112A04D1002900D03225290064
:10975000F2E7002D08D12000FFF732F9002803D0EE
:10976000102302791343037121002800FDF798FAB2
:10977000C2E7C0461468FF1F0C68FF1F1068FF1F78
:1097800070B50E4E8500AB590400002B13D01B782A
:10979000002B11D10A4B1B68002B04D05B68002BF7
:1097A00001D02000984773595B78122B03D1002118
:1097B0002000FFF7D9FE70BD024BECE71468FF1FD5
:1097C0001068FF1F0C68FF1F094B8000C358102052
:1097D000002B0CD01A6A002A09D09B68002B06D0F7
:1097E000127A1B7E101C9A4200D9181CC0B2704716
:1097F0001468FF1F70B503000D0014000220002A3A
:1098000030D000292ED013700B78081D53704B7880
:109810009370FFF7A7FCE070012002212B7A2371DF
:109820006B7B034063716A7B0A40134304226371BC
:109830006E7B1640334363716E7BF608F60033434C
:1098400063712B7B0340A371287B014000200B43F5
:10985000A371297B0A401343A3712A7BD208D2004B
:109860001343A37170BD10B50A0001000120FFF77A
:10987000C1FF10BD10B50A0001000220FFF7BAFFBA
:1098800010BD70B506000C000220002E30D000295B
:109890002ED07378201D0B70B3784B70F178FFF7E2
:1098A0006DFC01223579257271794B100800134047
:1098B000934010400343881010408000C9080343C0
:1098C000C9000B436373B1794B10080013409340F8
:1098D00010400343881002409200C9081343C90096
:1098E0000B4321202373FCF773FE854201D2122023
:1098F00070BD2220257AFCF76BFE8542F7D82378CD
:109900001820042BF4D86378012BF1D80020EFE75E
:10991000030010B50220002909D0002B07D0032234
:10992000481C0A7019000D3202F0E2F8002010BD48
:1099300003000222080010B5002B06D0002904D035
:109940000E32591C02F0D4F80022100010BD0300A2
:1099500010B50220002909D0002B07D00422481C92
:109960000A7019000C3202F0C3F8002010BD10B5C7
:10997000FFF7DEFF10BD03000220002906D0002BF8
:1099800004D0052200200A701B784B70704703003A
:109990000220002B08D0002906D05B7800200B7035
:1099A000013B082B00D918307047030010B5022086
:1099B000002909D0002B07D00622481C0A70190084
:1099C0000A3202F095F8002010BD10B5FFF7B0FF85
:1099D00010BD02000B00022010B500290ED0002A95
:1099E0000CD007211970118859701188090A9970D3
:1099F00011180822D81C02F07BF8002010BD0300CB
:109A00000A00022010B5002B0CD000290AD099784A
:109A10005878090201431180901CD91C082202F0D9
:109A200067F8002010BD030010B50220002909D0FE
:109A3000002B07D00822481C0A701900921802F067
:109A400057F8002010BD02000B00022010B50029BD
:109A50000BD0002A09D009211970117818185970F3
:109A6000511C062202F044F8002010BD10B5FFF78B
:109A70005FFF10BD02000B00022010B5002A09D0C4
:109A8000002907D05178197011180622581C02F0CD
:109A90002FF8002010BD030010B50220002909D0C6
:109AA000002B07D00A22481C0A701900063202F067
:109AB0001FF8002010BD10B5FFF73AFF10BD0200DF
:109AC0000B00022010B5002A06D0002904D018008F
:109AD0005178FFF753FB002010BDF0B585B017009B
:109AE0001E006A4606230500080091819380FEF758
:109AF000C0FC1324011E02900CD03800B047041E95
:109B000005D1280001A9FEF76FFA041E02D00298C1
:109B100001F096FE2800FFF701FA200005B0F0BD25
:109B2000F0B504008BB0019115000021102202A8AD
:109B300002F0E6F8334EA700B85900283CD0C3889D
:109B4000A34239D10378002B36D14278062A18D1A6
:109B500002000100553235310C3006ABFFF7A9FA8F
:109B6000002829D12000FFF72FFE020006A902A835
:109B700001F0BEFF200002A902F02AF801200BB07C
:109B8000F0BD816E002917D00B8A112A28D19D4281
:109B90000ED101981231093A01F03AFE012807D19D
:109BA000BB5920009D6EFFF70FFE29000200DEE783
:109BB00032212000FFF7D8FC2000FEF701FF061E2F
:109BC0001BD0416A002918D00B8AAB4215D108225C
:109BD0000198123101F01CFE01280ED1716A0AE0D1
:109BE0009D42E9D108220198123101F011FE0128AD
:109BF000E2D1BB59996E8A7EB9E7200001F058FF87
:109C0000BCE7C0461468FF1FF0B56B4D87007E5956
:109C100085B0337802900393002B00D087E0B368BF
:109C2000346A01937078062817D101221B7D1342F4
:109C300002D0217B114218D10222134202D0217B93
:109C4000114251D10422134203D0237B134200D08E
:109C50008BE0019B5A7DEB5991E007380428F8D836
:109C600001F0E6FF032E42678300B36E002B03D1A1
:109C70001C2001F065FEB066EB599C6E002C1CD0D8
:109C800010220021200002F03BF80298FFF79CFD13
:109C900001002000FFF72DFA01F0A2FE2082200033
:109CA00008211230FFF725FA0298FFF78DFDA07604
:109CB000EB592100D888FFF70FFC0822EB591CE074
:109CC000B36E002B05D01A00198AF0881232FFF704
:109CD0000DFC0222019B197DEB5911423DD0207BE6
:109CE00010423AD0073208E0F488FCF7DBFD0100AF
:109CF0002000FFF711FC0A22EB595A70029B9C00CE
:109D00002A595378073B042B11D8D088FEF758FE08
:109D100000284ED0C3895A08D2182849029B0298BD
:109D2000CB542B5941180433254801F0B1FD05B03F
:109D3000F0BDFCF79FFD03000120834201D100200C
:109D40000393EB59DE88FCF79BFD0399020030007A
:109D5000FFF7ECFB019AEB59117D042211420CD064
:109D6000217B114209D00B22C7E7F688FCF73CFDA6
:109D700001003000FFF7EEFB6BE7019A527D0121F5
:109D80000A4204D0607B084201D00C22B5E70221D0
:109D90000A4204D0607B084201D00E22ADE70421C4
:109DA0000A4204D0627B0A4201D01022A5E71222A7
:109DB000A3E7FA225200B0E71468FF1F1868FF1FDC
:109DC0007FA1001110B5064B1A780423100018402B
:109DD0001A4200D00348FFF727FA002010BDC04602
:109DE000A166FF1F2445FF1F70B50400FFF7D4FADA
:109DF000051E43D12000FFF77FFA234EA400A0598F
:109E00008268937CDB0708D50321036A1B790B402A
:109E1000012B02D1017F0B430377431DD97F8B1E9A
:109E2000022B0DD8022900D00121C088FCF790FF39
:109E3000042133591A7F59700A431A77280070BDDC
:109E400001290CD102231022437000210C3001F0B3
:109E500057FF305910213530FFF74BF9EEE7052950
:109E6000ECD10223D118437010220C3001F040FED7
:109E700004233259117F0B431377EAE7082518288A
:109E8000DCD1053DDAE7C0461468FF1FF0B58BB0A2
:109E9000059143887E4F9E00F45915000493002CD1
:109EA00015D1012902D000200BB0F0BD101D57784C
:109EB0001678FFF757F9EB68320002932B7A049972
:109EC000019300903B002000FCF70CFFEBE7E388D8
:109ED000049A934201D00820E6E72378012B00D1B1
:109EE000D4E0059B581E092800D9CFE001F0A0FE60
:109EF00005CE0A29CC506C859AB229000498FFF748
:109F000073FFD1E7200029001022453001F0F0FD59
:109F1000B9594B78042B02D1013B4B70C3E70B00BE
:109F20000A00253335320C310498FFF795F904986F
:109F3000FFF702FA0522431E9841BB59C0005A7030
:109F4000B2E7200029001022553001F0D1FD049B1A
:109F50004F4C9D00295904980A0006AB55320C312C
:109F6000FFF77AF929591022453106A801F050FC73
:109F7000012808D10498FFF7F7F90590002804D1CB
:109F800006222B595A7005988EE708230593FAE7A5
:109F900063780C2B7AD1E36E002B03D11C2001F0E7
:109FA000CFFCE066BB59D86E00286FD01022290084
:109FB00001F09EFDBB590498DC6EFFF705FC0D22F5
:109FC000A076BB595A706EE7E06E00285ED06378C9
:109FD0000D2B5BD12B8808220382A91C123001F0C3
:109FE00087FDBB599A68517D0222114226D0186A1A
:109FF000407B104222D00C32E4E763780E2B45D12F
:10A00000236F002B03D1162001F09AFC2067BB5967
:10A01000186F002803D01022290001F069FD0F22DB
:10A02000BB59CFE763780F2B30D1206F0622691C14
:10A03000103001F05DFDBB599A68517D0422114238
:10A0400003D0196A497B1142D5D100210498FFF74A
:10A050008BFA28E7636F002B0DD0BB59586F00288F
:10A06000F3D01022290001F043FD0122BB595242D6
:10A070005B6F1A61E9E7142001F062FCBB5960676D
:10A080005B6F002BE9D126E72978DFE707200BE794
:10A090001468FF1F10B5064C207001F0E9FD062181
:10A0A0002078FDF791FF0348FEF778FC10BDC0460D
:10A0B0002768FF1F3592001100200BB270B50D000C
:10A0C000834216DA264B187801F0C2FD041E0DD02B
:10A0D0000378922B0ED0A02B37D0224B1878FF2874
:10A0E0003AD0210001F0C4FC002835D180200002C4
:10A0F000684070BD43780E2B0BD03E2BEDD183789A
:10A10000052B12D0082BE8D181798088FFF7D8FA87
:10A1100008E0154B82889A42DFD183681878591C71
:10A12000FEF7C0FE002817D1D7E7104B1B785B075E
:10A1300012D50F4B1B68002B0ED09B68002B0BD049
:10A14000C289811D80889847ECE7FFF741FAA06833
:10A15000002801D001F074FB200001F009FDC5E7E3
:10A160002768FF1F1D45FF1F18200000A166FF1F65
:10A170001068FF1F10B50078FFF712FA10BD10B578
:10A180000078FFF7FDFA10BD0C234343084A10B5D1
:10A190009B185A68002A03D0012901D1904710BDAD
:10A1A0009B68002BFBD00029F9D19847F7E7C04600
:10A1B0004468FF1F01238340094A10B5946B1C4378
:10A1C0009463506B98435063D46B200098430129EB
:10A1D00001D120001843D063116B0B43136310BDF2
:10A1E00000800040F0B500240127154B85B0DA6BE4
:10A1F000144E03921A6C0192DA64019BE3403B42D5
:10A2000017D0039DE5403D400295E5B20299280034
:10A21000FFF7BAFF316A736A002908D03900002BB2
:10A2200001D0029979402800FFF7C4FF01E0002B1C
:10A23000F9D101340C36172CDFD105B0F0BDC04682
:10A24000008000402868FF1F064B01215A68C24069
:10A250000A4204D01B68C3401800084070471B6DB9
:10A26000F9E7C046008000400122064B82400029E9
:10A2700003D0D9680A43DA607047D9689143D9603E
:10A28000FAE7C0460038004030B5032444430F4B82
:10A29000E25C1B199C785D7801232D1B0135AB40D6
:10A2A000013BA340A140DB430C00122807D808491A
:10A2B00092005218116819402143116030BD054ABF
:10A2C00011680B4023431360F8E7C04607C0001134
:10A2D00008F0004014F00040C21F70B5D4B206234D
:10A2E000092C0BD80125084C9540002908D00021E5
:10A2F000FFF7CAFF23682B4323600023180070BDBB
:10A300002368AB43F8E7C04600380040214BF0B566
:10A310001B185B78022B21D1032444431E4A1F4E95
:10A32000A35C12199478012215008540B76B013C9B
:10A33000E4B23D43A240B563194C122815D89B00E6
:10A3400000290CD117495B1899680A439A600123C8
:10A35000205C154A834011680B431360F0BD11491E
:10A360005B18996891439960F1E70E4B00290DD174
:10A3700059690A435A61225C1328E8D00123203A24
:10A3800093400A49086803430B60E7E75969914322
:10A390005961F0E72868FF1F07C0001100800040E6
:10A3A0004CC0001100F00040A0F00040A4F00040BC
:10A3B000F8B500241B4E1C4D1C4B1B5D012B1FD1FF
:10A3C000194A9269E2401A420BD00122B2569340D8
:10A3D0002200143AD2B2022A09D815494A69134315
:10A3E0004B61013402360C35172CE5D1F8BD002243
:10A3F000B2560F499200521891680B439360F0E7F0
:10A40000022BEED1E7B23800FFF71EFF01235840C0
:10A41000C1B23800FFF77AFF3800FFF715FF687701
:10A42000DFE7C046D9BF00112868FF1F2968FF1F5A
:10A4300000F00040012202388240054B002903D081
:10A4400059690A435A617047596991435961FAE75A
:10A4500000380040F8B50E0001210F008740114A76
:10A460000400D368FD43BB43D360831E8B4201D8F5
:10A47000FFF7E0FF00212000FFF72EFF0A4A0B4BF9
:10A480005168012E05D139431B1951605E700020BF
:10A49000F8BD2940516002221C1962709A6915406A
:10A4A0009D61F4E700380040008000402868FF1FED
:10A4B000012210B58240074B002906D019680A43D3
:10A4C0001A600121FFF7C6FF10BD1968914319609A
:10A4D000F7E7C046008000400C2370B500254343D9
:10A4E0000A4A29009B181D70094B04001B185D7057
:10A4F000FFF7B0FF0123A340064928000A681A436A
:10A500000A6005490A689A430A6070BD4468FF1FE3
:10A510002868FF1F348000403080004070B5040080
:10A520000E00FF2813D003250540FFF7D5FF084A8A
:10A53000A3089B009B183F22ED00AA40AE4019687B
:10A5400020009143314319600121FFF78DFE70BD5A
:10A5500018380040F8B50C244443134B0500E418A8
:10A560006368002B03D1A3681220002B1AD00222AB
:10A5700001270E4B00215B195A7028002770FFF746
:10A5800069FF63681E1E08D0A3683E00002B04D03C
:10A590002800FFF759FE4640F6B228003100FFF7C9
:10A5A00009FE0020F8BDC0464468FF1F2868FF1F51
:10A5B000F7B5C420FF222B4B80001958002491438B
:10A5C0003F3A0A431A508022274F5202274E1A6000
:10A5D000274B1D5D002D21D0A31E012B03D8012187
:10A5E000E0B2FFF727FF012D18D11F4B9B69E34015
:10A5F0002B4213D0E3B218000193FFF725FE0100B0
:10A600000198FFF755FFE3B2143B022B1DD801213F
:10A610007156184A8D405369AB4353613B7F002B01
:10A620000DD0E5B22800FFF795FF2800FFF70CFEDC
:10A630007B7F0100834202D02800FFF7A5FD013493
:10A640000C370236172CC3D1F7BD012100237156F8
:10A65000F3568D40074A9B009B189A68AA439A605C
:10A66000DCE7C04600E100E02868FF1FD9BF001109
:10A670002968FF1F00F0004070B50E0015000400AF
:10A68000FFF72AFF0C236343094A20009B189D60B3
:10A690005E60FFF75FFFF021064B074A8900051E49
:10A6A0005A5002D02000FFF717FF280070BDC046A7
:10A6B0004468FF1F0000FF1FE5A1001170B5134D96
:10A6C00007202C78002C1FD198222100520028004E
:10A6D00001F076F80123C420FF222B700C4B800080
:10A6E0001C635C630B4B1C605C600B4B1958914303
:10A6F0003F3A0A431A50802252021A600D20074A3C
:10A70000074901F015F9200070BDC0462868FF1FF9
:10A7100000800040A0F0004000E100E0B1A5001181
:10A72000B1A30011030010B50620072B09D8054A74
:10A73000137001F09DF8D7210020034B034A8900D4
:10A740005A5010BD4C45FF1F0000FF1F151BFF1F77
:10A7500070B51D0002240C2910D8094ACA40D2073E
:10A760000CD5FBF741FF041E08D1059A0499280077
:10A77000FBF756FFFCF7C4FDFFF724FB200070BD7C
:10A780001210000030B50D7802232C009C431842B3
:10A7900001D02B431C0008252300AB43284201D0E5
:10A7A0002B00234320241D00A543204201D01C433D
:10A7B00025002A230D70184204D011781E3B0B434C
:10A7C000137030BD0028FCD10C2113788B43F7E7C0
:10A7D000F8B51D0006AB1B88140007AA0E000B205D
:10A7E0001778002B27D10A78022A49D14A68507875
:10A7F00011780002244A08438018042840D801F048
:10A8000017FA03121D1B2300F06800F081FF021CE1
:10A81000C0B2B84200D93A1CD2B22000F1682A80F6
:10A8200001F066F906E00222F3681B882A80237093
:10A830001B0A63700020F8BD0622EEE701232B807F
:10A84000F3681B782370F5E7F368002B16D0082215
:10A850002A801A8822701A88120A62705A88A27096
:10A860005A88120AE2709A8822719A88120A6271D2
:10A87000DA88A271DB881B0AE371DBE72B80D9E75A
:10A8800001202B80D7E7C04600D6FFFFF7B51600A2
:10A890000A781D0008AB1F880C000123022A18D17A
:10A8A0004A685078117800022B4A08438018032820
:10A8B0000FD801F0BDF902254439E06800F028FF07
:10A8C000C0B20723B84204D37B190193152B02DDD4
:10A8D0000D231800FEBDE0682A003100C01901F008
:10A8E00007F96B4600209B88E268D0541B4B1B681D
:10A8F000834203D01B68834200D098470023E8E7D7
:10A900000B23002FE5D1022DE2D1737832781B02A0
:10A910001343E2681380114B1B68002BEED01B68B9
:10A92000002BEBD00120E8E70B23002FD1D1062D1F
:10A93000CED12A003100E06801F0DAF8DEE70B231F
:10A94000002FC6D1012DC3D132787533012AC0D86A
:10A95000E3681A70D2E7C04600D6FFFF346AFF1FD3
:10A9600070B50C001500072837D801F061F9041400
:10A9700036361B36242E182015290BD8184E1622D1
:10A980000021300001F0BCF922002900300001F064
:10A99000AFF8002070BD18200229FBD11288114B9E
:10A9A0001A80F6E718200829F4D10A000E48290079
:10A9B00000F016FFEDE718200129EBD10B4B1078C2
:10A9C0000B49DA69FFF7DEFEE3E718200129E1D140
:10A9D000064B10780749DA6BF4E70220DAE7C04645
:10A9E0001C6AFF1FCA45FF1FC045FF1F5045FF1FC0
:10A9F0007845FF1F9845FF1F030010B50020DB07B7
:10AA000004D50721024A034800F08CF810BDC04667
:10AA100064C000115045FF1F054A0300106800285C
:10AA200003D082889A4201D1806870470068F6E7B7
:10AA3000386CFF1F0A88030008009A4204D08A88F5
:10AA400004309A4200D0002070470000F8B5F82288
:10AA500000230D4F0D4E7968050042433370994233
:10AA600000D07B600A4C0021200001F049F900234E
:10AA70001A007C60AB4202D100203370F8BD013374
:10AA80002280DBB2F834F5E7386DFF1F346DFF1F0D
:10AA90003C6CFF1F73B56B460190060068461500BD
:10AAA0001980FCF75FFF041E11D1002D0FD07689AD
:10AAB000002E11D00C2000F043FF00280ED0084AD1
:10AAC0000460136886808560002B02D1106020002E
:10AAD00076BD1A001B68F7E70224F8E71324F6E7AF
:10AAE000386CFF1F012100220A4B10B549420A4C65
:10AAF000198099809A719A70084B207001201980F2
:10AB00005A60FFF7A3FF2078FCF78AFF0448FDF79F
:10AB100045FF10BD3C6AFF1F406DFF1F386DFF1FD2
:10AB2000D1AB0011022310B5002802D0FFF7B2FF0D
:10AB30000300180010BD0000030010B50020DB0763
:10AB400004D50421024A0348FFF7A4FF10BDC04604
:10AB500078C00011D045FF1FF0B50E2687B00393D3
:10AB60000CAB1F8802ABF6180500080031000292FA
:10AB7000FDF77AF804000120002C0FD03088FFF791
:10AB80004BFF03000E20002B08D05E68002E05D07E
:10AB900021002800039B029A0097B04707B0F0BD40
:10ABA0000A4B10B5984207D10122002352420A8075
:10ABB0008B708A808B7110BDFFF73CFF0028FAD0A4
:10ABC00001235B42038000238370F4E7FFFF000052
:10ABD000F8B5050001290AD1134E00243388F8275F
:10ABE000AB4219D028001149FFF7DAFF06E002292D
:10ABF00004D10139FDF750FF0028EDD0F8BD3B002E
:10AC000063437268D018D35A002B09D03A00002150
:10AC100001F076F80134E4B2054B1B78A342EED87C
:10AC200001235B423380DDE7386DFF1F3C6AFF1F65
:10AC3000346DFF1F10B5FFF7FDFE030000208342B7
:10AC400000D0987810BD0000F0B589B01C000EABA4
:10AC500080CB03901E8810AB1B78049202930B7A72
:10AC60000D00DB0616D42B780593022B24D0049814
:10AC7000FFF7D2FE002812D003689C46002B0ED0AE
:10AC8000029B2200019329003B0064460398009632
:10AC9000A04705E00498FFF7BFFE002802D10E2070
:10ACA00009B0F0BD8368002BF9D00A22290003986F
:10ACB00098470028D7D0F3E76B6858781A786B4B21
:10ACC000000210439842D2D8043B984210D2684BFD
:10ACD000984242D015D8674BC0180128C7D80B201E
:10ACE000002EDDD1EB681A7859683A80200028E000
:10ACF000614BC018032800D979E000F099FF846AFD
:10AD0000789E5E4B9842B2D10B20002EC8D1012311
:10AD10003B80EB6831001B7823706889013080B27A
:10AD2000FCF7A2FF3A88031E0ED0017802328A187F
:10AD30003A80428962704289120AA2705968027888
:10AD4000E01C00F0D5FE06E004323A803100042217
:10AD5000601C00F0D5FF0020A2E70B20002E9FD141
:10AD6000EB6807A91E8804233B80330A3000267055
:10AD70006370FCF779FF051E28D004AB9A890E2377
:10AD800004A95B183E49C668FCF7E2FF00280BD116
:10AD90002B783C486A680599FBF798FB002803D19B
:10ADA000012304AA5B42D3813278022A06D171685A
:10ADB000201D00F09DFE3B8802333B800E2304AA39
:10ADC0009B181B88A3701B0AE370C4E704ABDE81E9
:10ADD000F4E70B20002E00D062E7E9680398FFF744
:10ADE00029FF02233B802070000A6070B3E70B202C
:10ADF000002E00D054E70222EB681B883A802370B3
:10AE00001B0A6370A7E7E86800F082FCC2B2030087
:10AE10000720B24200D243E70DD00299DBB271188D
:10AE2000994202DB921BD3B20293029BE9681A009B
:10AE30003B8089195AE70023F6E70B20002E00D04B
:10AE40002EE70722EB683A801A7822705A786270EF
:10AE50005A88A2705A88120AE2701A792271DA8826
:10AE60006271DB881B0AA37175E7C04604290000E4
:10AE70000228000000D8FFFFFFD6FFFF03280000D4
:10AE8000FFFF0000A8BF0011F0B58DB06B46002099
:10AE9000089120229B5E83423DDAA64B187800F091
:10AEA000D7FE071E32D00378B02B2CD100790238A0
:10AEB00016281FD800F02CFD17001E001E001E00D3
:10AEC00031001E0096001E001D011E0052011E00D2
:10AED00073011E00CD011E0050021E001E001E0048
:10AEE0008E021E00E302944B94491B8878880B80E5
:10AEF000FBF72CF83800FCF7ADFF914B1B68002BDB
:10AF000001D038009847380000F032FE8020089BBE
:10AF10000002434018000DB0F0BDF6220021874822
:10AF200000F0EEFE0BAA3B7B7989388900923A004B
:10AF30000D32FCF7B1FD0400804B1B78002C3FD193
:10AF400046E0804B788805937F4B4100CB5A0BAE8F
:10AF5000073BDBB232880293002301937B4B210035
:10AF600006930093059BFFF76FFE744D002810D1E8
:10AF7000069B3A8A1B889A420BD1380005991230F9
:10AF800000F046FC002804D02B7862899B00EB1867
:10AF90005A80162306A81B18328820007989FCF7EE
:10AFA000D7FE2B7804009A00AA1851880029C3D034
:10AFB0000133DBB22B70002807D006A9C98A918023
:10AFC000634A12889A42BCD802E00121494291802A
:10AFD000002B04D059497888FAF7ECFF8AE73E89BC
:10AFE0000A2479E000253E89574B06937B88069A10
:10AFF0005B009B5A033B9D4202DB002DF0D05BE0DF
:10B00000162206A812183B7B798900923A0030007C
:10B010000D32FCF741FD0590002858D04689017A91
:10B020007888FCF703FD041E44D1464B78880793CB
:10B03000069B4100C95A454B0439C9B206AAD28AB7
:10B0400006930291019400930599079BFFF7FCFD7D
:10B05000041E2FD1069B39491A88931C002D26D136
:10B060004B807988384B4900CB5A5119033B8B42AE
:10B0700020DD059B31485B8941190B71A91C013505
:10B08000C9B2EDB2059145191B0A2B71059B2D49DB
:10B090000433181800F02CFD2C4B059A1B88D3188C
:10B0A000DDB22C4B9E4205D00136B6B29CE74988F2
:10B0B0009942D6D0002D0CD0204C2800618800F099
:10B0C0007FFD207021007888FAF784FF12E7059C45
:10B0D000F0E7002C00D183E77B78142B00D109E73F
:10B0E00016493B794E800B700C717888FAF724FF73
:10B0F00000E7162406ABE41821003889FCF7B4FDFC
:10B10000011E00D1B7E1788822880F4C45002C5BE6
:10B110000A4D013CE4B2029400240F4B01940095C7
:10B12000FFF792FD041E00D014E129007888FAF799
:10B1300061FFDFE6406DFF1FBC44FF1F446AFF1F35
:10B14000386AFF1F3E6BFF1F7466FF1F346CFF1FC2
:10B15000BA44FF1FFFFF0000466AFF1F162406AB1C
:10B16000E41821003889FCF77FFD011E00D182E13F
:10B1700078882288AE4C45002C5BAE4D013CE4B291
:10B1800002947C89AC4B01940095FFF75DFD041E91
:10B1900000D0DFE029007888FAF736FFAAE600251C
:10B1A000A44B1D803B00FE331B78A24A788807928F
:10B1B000AB4208D99E4B12880693069943005B5A0E
:10B1C000013B9A4203DB0799FAF728FF92E616241F
:10B1D0006B00FB18059306ABE418059B210018894A
:10B1E000FCF742FD011E03D1059B01241E8973E774
:10B1F0007888924B2288069C099343001B5B904EF3
:10B20000013BDBB20293002300960193099BFFF7F9
:10B210001BFD041E02D0059B1E895DE77B88069AF4
:10B220005B009B5A079A108832881218934202DCFE
:10B230001B1A013B33807F4C023032880999001978
:10B2400000F056FC2388328801359B182380EDB22C
:10B25000A8E70BAA3B7B7989388900923A000D3226
:10B26000FCF71AFC00250590059B002B04D10A244D
:10B27000002D00D16EE060E0059B7888197AFCF71C
:10B28000D5FB0100041E63D1694C6C4B7888069491
:10B290000993069B4400E45A694B063CE4B20BAEAA
:10B2A000328807930294019100930599099BFFF757
:10B2B000CBFC041E4CD1079B5E491B881A1D002D38
:10B2C00030D14A80059B5B4C5A8963191A716B1CFB
:10B2D0009BB2E318120A1A71162306A832881B18AB
:10B2E00079890598FCF734FDFF21AA1C2E1D033532
:10B2F0000B00059092B2B6B2ADB2002803D006ABF7
:10B30000DB8AD9B21B0AA218651911712B714C4D39
:10B31000301D2A884949201800F0EAFB2B88F618CE
:10B32000B5B2A1E74988914207D17A8806995200BF
:10B33000525AEB18053A9A42C4DC3E4C2800618808
:10B3400000F0D6F9207021007888FAF771FED1E577
:10B35000002DF2D13E89BFE6162606ABF618310065
:10B360003889FCF781FC3D000400FF3500282DD012
:10B37000037A9B060CD400227B8939897888009255
:10B380003A000C32FFF7E8FB041E10D03E8915E0AE
:10B390003088FFF741FB00281AD08368002B17D0B4
:10B3A0002100122278889847041EE4D0EEE7AB789B
:10B3B000002B02D17888FAF74BFE0026AB78002BE1
:10B3C00000D097E5002C00D194E585E60124DDE767
:10B3D0000E24DBE7162506ABED1829003889FCF7AB
:10B3E00043FC041E47D0037A9B0611D4154A7B8880
:10B3F0001188994203D01448814207D11380134B1E
:10B40000F8261D780023D9B2A94221D30924A1E747
:10B410002888FFF701FB00282FD08368002B2CD051
:10B420002100122278889847041EDFD092E7C04698
:10B430007466FF1F446AFF1F466AFF1F3E6BFF1FB3
:10B44000346CFF1F386DFF1FFFFF0000346DFF1FBE
:10B4500031005943546801336018615A0029D2D130
:10B460003C0008342100F82200F042FB21007888DB
:10B47000FAF7F6FD3EE501246CE70E246AE71D4B62
:10B480001A887B889A4231D07888FAF7F3FD31E543
:10B49000F823059851684343CD18C95A00291FD095
:10B4A0003B7A012B0BD16C88AB887888AA1D00945D
:10B4B000FFF752FB041E02D000233B722E88F822B5
:10B4C0000021280000F01CFC00232B80059B013389
:10B4D000DBB20593084B05991B78064A8B42D7D8F7
:10B4E00001235B421380002CCED0F5E5002634000A
:10B4F0000596EFE7386DFF1F346DFF1F70B5040030
:10B500000E001500FFF796FA031E08D1310005481A
:10B51000FFF790FA03001120002B02D01C800020BE
:10B520009D7070BDFFFF0000F8B50B4F06003B7823
:10B530000D001400FF2B0ED00A2000F071FB011E3D
:10B5400009D0B1230380002346800371C5800481A4
:10B55000387800F08DFAF8BD1146FF1FF7B50F00DF
:10B5600008A90600088809A90B240988002821D108
:10B570000234022B1ED1557813782D021D432B0067
:10B580008B4301937334002B14D1FB6830001900F6
:10B590000093FFF74FFB019C85420BD02A0030003F
:10B5A0000099FFF7ABFF041E04D12A00300079890F
:10B5B000FFF7BAFF2000FEBDF0B50E7885B003900E
:10B5C0000AA805880120022E0DD14C6827786478DE
:10B5D00024023C43054FBC4205D10398DBB20196DF
:10B5E0000095FFF7BBFF05B0F0BDC0460229000083
:10B5F00010B504000C4800F003FB0C48A16B00F0F0
:10B60000FFFA0B48E16B00F0FBFA0A48216C00F0EE
:10B61000F7FA094B0948196800F0F2FA084B1B6861
:10B62000002B00D09847FEE75ABE001170BE0011F3
:10B630007FBE00118EBE001104ED00E09DBE001122
:10B64000446DFF1F002307B501A80193FFF7D0FF4A
:10B65000044A0548002110B5121A00F051FBF8F712
:10B66000AFF9FEE7486DFF1F1446FF1F0000000002
:10B6700001B40248844601BC604700BFB14E0000DF
:10B6800001B40248844601BC604700BFF539FF1F82
:10B6900001B40248844601BC604700BFB54C0100BC
:10B6A00001B40248844601BC604700BFE139FF1F76
:10B6B00001B40248844601BC604700BF3555000014
:10B6C00001B40248844601BC604700BFEDA50000FC
:10B6D00001B40248844601BC604700BFC53F00007A
:10B6E00001B40248844601BC604700BFC95C010048
:10B6F00001B40248844601BC604700BF090E000047
:10B7000001B40248844601BC604700BF851F0000A9
:10B7100001B40248844601BC604700BFDD5201000D
:10B7200001B40248844601BC604700BFC521000047
:10B7300001B40248844601BC604700BF5D170000A9
:10B7400001B40248844601BC604700BFC13BFF1FF3
:10B7500001B40248844601BC604700BF017F00007D
:10B7600001B40248844601BC604700BF9DA90000A7
:10B7700001B40248844601BC604700BF2D35FF1F5D
:10B7800001B40248844601BC604700BFA532FF1FD8
:10B7900001B40248844601BC604700BFE548000090
:10B7A00001B40248844601BC604700BF7530FF1FEA
:10B7B00001B40248844601BC604700BF6DBC000074
:10B7C00001B40248844601BC604700BFB70E0000C8
:10B7D00001B40248844601BC604700BF953BFF1F8F
:10B7E00001B40248844601BC604700BF810E0000DE
:10B7F00001B40248844601BC604700BFED4A010025
:10B8000001B40248844601BC604700BF2539FF1FD0
:10B8100001B40248844601BC604700BFCD4C010022
:10B8200001B40248844601BC604700BFC51D00004A
:10B8300001B40248844601BC604700BF55220000A5
:10B8400001B40248844601BC604700BFD9490100E9
:10B8500001B40248844601BC604700BF5125000086
:10B8600001B40248844601BC604700BF1D4B010083
:10B8700001B40248844601BC604700BF151BFF1F8E
:10B8800001B40248844601BC604700BF7138FF1F05
:10B8900001B40248844601BC604700BFA9460100CC
:10B8A00001B40248844601BC604700BF0D5201004C
:10B8B00001B40248844601BC604700BF8B520100BE
:10B8C00001B40248844601BC604700BF014C01003E
:10B8D00001B40248844601BC604700BF7D37FF1FAA
:10B8E00001B40248844601BC604700BF291C000027
:10B8F00001B40248844601BC604700BFD91B000068
:10B9000001B40248844601BC604700BF055E0000E8
:10B9100001B40248844601BC604700BFE53CFF1FFC
:10B9200001B40248844601BC604700BFE92800001A
:10B9300001B40248844601BC604700BFED32FF1FDE
:10B9400001B40248844601BC604700BF3D4B010082
:10B9500001B40248844601BC604700BF4D32FF1F5E
:10B9600001B40248844601BC604700BF6D3AFF1F26
:10B9700001B40248844601BC604700BF2146010073
:10B9800001B40248844601BC604700BFF94C010085
:10B9900001B40248844601BC604700BFE1170000C3
:10B9A00001B40248844601BC604700BF7D18FF1FF8
:10B9B00001B40248844601BC604700BF55490100FC
:10B9C00001B40248844601BC604700BF1147010032
:10B9D00001B40248844601BC604700BFA137FF1F85
:10B9E00001B40248844601BC604700BF29510100F0
:10B9F00001B40248844601BC604700BF8D120000BC
:10BA000001B40248844601BC604700BF350E000007
:10BA100001B40248844601BC604700BF1D36FF1FC9
:10BA200001B40248844601BC604700BFC94A010016
:10BA300001B40248844601BC604700BF3D180000C5
:10BA400001B40248844601BC604700BFADAE0000AF
:10BA500001B40248844601BC604700BFC130FF1FEB
:10BA600001B40248844601BC604700BF4551010053
:10BA700001B40248844601BC604700BF594F010031
:10BA800001B40248844601BC604700BF5147010031
:10BA900001B40248844601BC604700BFBD3CFF1FA3
:10BAA00001B40248844601BC604700BFCD34FF1F8B
:10BAB00001B40248844601BC604700BF091B000076
:10BAC00001B40248844601BC604700BF65710100B3
:10BAD00001B40248844601BC604700BF2D3AFF1FF5
:10BAE00001B40248844601BC604700BFC9A90000F8
:10BAF00001B40248844601BC604700BFE94C010024
:10BB000001B40248844601BC604700BFAD3AFF1F44
:10BB100001B40248844601BC604700BF75A900001B
:10BB200001B40248844601BC604700BF4D1F0000BD
:10BB300001B40248844601BC604700BF456B010068
:10BB400001B40248844601BC604700BF01240000E4
:10BB500001B40248844601BC604700BF7918000068
:10BB600001B40248844601BC604700BF5118FF1F62
:10BB700001B40248844601BC604700BF434D010048
:10BB800001B40248844601BC604700BFDD66010085
:10BB900001B40248844601BC604700BF252600006E
:10BBA00001B40248844601BC604700BF59520100FD
:10BBB00001B40248844601BC604700BFB352010093
:10BBC00001B40248844601BC604700BF350E000046
:10BBD00001B40248844601BC604700BF311B00002D
:10BBE00001B40248844601BC604700BF8D34FF1F8A
:10BBF00001B40248844601BC604700BF2124000014
:10BC000001B40248844601BC604700BFE53A010028
:10BC100001B40248844601BC604700BFA54F010043
:10BC200001B40248844601BC604700BF1D4D0100BD
:10BC300001B40248844601BC604700BFD13CFF1FED
:10BC400001B40248844601BC604700BFF30E000007
:10BC500001B40248844601BC604700BFF54E0100B4
:10BC600001B40248844601BC604700BFC56D0100B5
:10BC700001B40248844601BC604700BFC9260000E9
:10BC800001B40248844601BC604700BF4550000033
:10BC900001B40248844601BC604700BF090E0000A1
:10BCA00001B40248844601BC604700BF691F000020
:10BCB00001B40248844601BC604700BF056A000029
:10BCC00001B40248844601BC604700BF85520100B0
:10BCD00001B40248844601BC604700BF6532FF1FC3
:10BCE00001B40248844601BC604700BF193BFF1FF6
:10BCF00001B40248844601BC604700BF156B0100D7
:10BD000001B40248844601BC604700BF154D0100E4
:10BD100001B40248844601BC604700BF01890000AD
:10BD200000030102020303030403050006020700E7
:10BD3000080209030A030B030C000D000E030F0396
:10BD4000100311031203130314031502160200005B
:10BD50009D3D0011D13D00110000000002000000D7
:10BD600066BD0011192A0F180A000000F1590000E1
:10BD7000FD24000041460100A5800011B9A000117A
:10BD80000D750011A97E00118153001189AE0011BB
:10BD9000E94F0011953F0011C5400011000000005F
:10BDA0001616000002000000B0BD0011F4FFF3FF02
:10BDB000D2FC00000542001100000000000000005D
:10BDC000547579610042312E3300303031370067CD
:10BDD00069746875622E636F6D2F70767678005483
:10BDE0004842310002000000F8BD0011292A282A2B
:10BDF000272A262A252A242A0A180000E2040000FD
:10BE00007102000078EC0000744000001027000070
:10BE100060F0000006640000204E000000000000FA
:10BE2000050000001F501D00023CB4000001170077
:10BE300013000000A10200003031323334353637B0
:10BE40003839414243444546005048592B36325810
:10BE500058504C555330353034005B486172642083
:10BE60006661756C742068616E646C65725D0A0051
:10BE70004C522020203D203078253038780A005060
:10BE8000432020203D203078253038780A00505358
:10BE90005220203D203078253038780A004943531D
:10BEA00052203D203078253038780A00855700111F
:10BEB000D95700110000000002000000C4BE0011AC
:10BEC0006F2A6E2A1A18EAD8BC80F0FC60000000C5
:10BED0000000000000005F066B2F363D7D077F3FAE
:10BEE000777C596E7971000001A00000000000000D
:10BEF0006410B71DC8206E3BAC30D9269041DC766B
:10BF0000F4516B6B5861B24D3C7105502083B8ED14
:10BF100044930FF0E8A3D6D68CB361CBB0C2649B38
:10BF2000D4D2D38678E20AA01CF2BDBDFB349B5F5D
:10BF30008000008000100000000000000F61001170
:10BF40009977001133610011A17B0011B7610011D5
:10BF5000777B00112D6200114D7B00117F62001173
:10BF6000157D0011E7620011157D001119630011A4
:10BF7000CF7C00112D620011057B0011A56200111C
:10BF8000AD7C001100000000000000008B63001178
:10BF9000AD7C0011ED630011B1770011052A042A70
:10BFA000012A002A02290328012800280118001864
:10BFB00000000000000000000000000000000087FA
:10BFC0000101020102010102010203030401030154
:10BFD000010101010303020103000D000E00100026
:10BFE000110013001401070108010A010B011C01D3
:10BFF0001D02040205020702080219021A021C02AD
:10C000001D030103020317000201000504000807D5
:10C01000000B0A001716001D1C0102010105040196
:10C020000E0D011110011413011716011A19020245
:10C0300001020B0A020E0D02111002141302171650
:10C04000030504030807030B0A030E0D0001020396
:10C0500007090A0B0E0F101112141718191A1B1FBB
:10C0600020212200D1A700118DA80011000000009E
:10C0700002000000AEBF001100000000B9B50011C1
:0CC080000000000002000000ACBF001136
:020000041FFFDC
:1000000000000000F93E00116CBD001168BD001138
:100010002063FF1F0000000000000000000000003F
:1000200000000000000000000000000000000000D0
:1000300000000000000000000000000000000000C0
:1000400000000000000000000000000000000000B0
:1000500000000000000000000000000000000000A0
:100060000000000000000000000000000000000090
:100070000000000000000000000000000000000080
:100080000000000000000000000000000000000070
:100090000000000000000000000000000000000060
:1000A0000000000000000000000000000000000050
:1000B0000000000000000000000000000000000040
:1000C0000000000000000000000000000000000030
:1000D0000000000000000000000000000000000020
:1000E0000000000000000000000000000000000010
:1000F0000000000000000000000000000000000000
:1001000000000000000000000000000000000000EF
:1001100000000000000000000000000000000000DF
:1001200000000000000000000000000000000000CF
:1001300000000000000000000000000000000000BF
:1001400000000000000000000000000000000000AF
:10015000000000000000000000000000000000009F
:10016000000000000000000000000000000000008F
:10017000000000000000000000000000000000007F
:10018000000000000000000000000000000000006F
:10019000F134FF1F3933FF1FC1660100000000006A
:1001A000000000000000000000000000000000004F
:1001B000000000000000000000000000000000003F
:1001C000000000000000000000000000000000002F
:1001D000000000000000000000000000000000001F
:1001E000000000000000000000000000000000000F
:1001F00000000000000000000000000000000000FF
:1002000000000000000000000000000000000000EE
:1002100000000000000000000000000000000000DE
:1002200000000000000000000000000000000000CE
:1002300000000000000000000000000000000000BE
:1002400000000000000000000000000000000000AE
:10025000000000000000000000000000000000009E
:10026000000000000000000000000000000000008E
:10027000000000000000000000000000000000007E
:10028000000000000000000000000000000000006E
:10029000000000000000000000000000000000005E
:1002A000000000000000000000000000000000004E
:1002B000000000000000000000000000000000003E
:1002C000000000000000000000000000000000002E
:1002D000000000000000000000000000000000001E
:1002E000000000000000000000000000000000000E
:1002F00000000000000000000000000000000000FE
:1003000000000000000000000000000000000000ED
:1003100000000000000000000000000000000000DD
:1003200000000000000000000000000000000000CD
:1003300000000000000000000000000000000000BD
:1003400000000000000000000000000000000000AD
:10035000000000000000000000000000000000009D
:10036000000000000000000000000000000000008D
:1003700045B6001100000000000000000000000071
:10038000000000000000000000000000000000006D
:10039000000000000000000000000000000000005D
:1003A000000000000000000000000000951AFF1F80
:1003B000000000000000000000000000000000003D
:1003C000000000000000000000000000000000002D
:1003D000000000000000000000000000000000001D
:1003E000000000000000000000000000000000000D
:1003F00000000000000000000000000000000000FD
:081838005071FF1F4118FF1F52
:10184000024981F3088802F097FC00005071FF1FE5
:1018500010B502F069FC072804D0122808D002282D
:1018600008D010BD044A0420136B01331363F8E75A
:101870000220F6E71420F4E71C67FF1FF8B5070005
:101880000C0026002500503630785135002804D150
:101890000300287058342370F8BD2978CA00481E08
:1018A0008141A3183800A25C5B68C9B2FFF7D0FF82
:1018B00000280DD12B78DA00A218013350602B706C
:1018C0003378044A013B3370136A01331362D8E75B
:1018D0000123DFE71C67FF1F5C234343074910B563
:1018E000C9180B0058331B78012B05D1FFF7C6FF31
:1018F000034A936A0133936210BDC0465067FF1FCD
:101900001C67FF1F10B502F047FC064A01211300B7
:1019100010CB4942D967044B136002F0FDFA200056
:1019200010BDC04600E100E01000100010B504003A
:1019300002F032FC024B1C6002F0EEFA10BDC04611
:1019400000E100E010B5040002F026FC4021094A45
:10195000200013688B43136002F046FA01F0AAFDE1
:101960000022054B01201A60044B04321A6002F079
:1019700063FBFEE71CF00040C4F00040C0F00040F4
:10198000431E5A425341A022F0B5D2015B4213409C
:10199000154D164A40019B182A18127E8BB00191F2
:1019A000002A1BD01A000832D46F0022E6B206AF1C
:1019B000E4B294420EDC2818C369002B08D00199C8
:1019C00002AA117106AA049202AA167303A89847E4
:1019D0000BB0F0BD1978B9540132EAE71A7D1A78D4
:1019E00006AB01261A70E6E7DC69FF1F00400040E5
:1019F000F0B5254B04004001C25C85B0002A2BD015
:101A00001A18117E002927D0917E002924D011793F
:101A1000022921D11689D788D168F51BADB22A1CBD
:101A2000102D00D9102292B2BE4217D118180123EE
:101A300003710023C269C38003819A4206D06846BD
:101A4000032103730171029301A890470820002C21
:101A500000D0192001F026FC05B0F0BD013C654224
:101A60006C41A0256442ED012C40084D1B186419FF
:101A7000074D0633013A92B2AA42EDD01888461CAF
:101A80001E80085C2070F5E7DC69FF1F0040004005
:101A9000FFFF00000F220E4B10B59868104002386F
:101AA0000A280BD802F014F90D0A0B0A0A110A0AC7
:101AB0000A0A060002210020FFF762FF10BD012183
:101AC000F9E70020FFF794FFF8E7DB6FF6E7C04681
:101AD000004000400F220E4B10B5986810400238AD
:101AE0000A280BD802F0F4F80E0A0B0A0A120A0AA6
:101AF0000A0A060002210120FFF742FF10BD012162
:101B00000800F9E70120FFF773FFF7E7DB6FF5E760
:101B10000090004013B5334C2378072B3DD8324B4F
:101B20001A78324B002A39D18022196852020A43AE
:101B30001A60252001F07AFF20232D4A11680B43FB
:101B4000802113606B460422C905086807331042E0
:101B500028D080210422C905C86810422ED08021D7
:101B60002020C905CA688243CA6014221A701A78F4
:101B7000002A2FD18021C905C86820320243CA60DB
:101B800014221A701A78002A28D11A4B1A7D22784A
:101B90005A601D221A705932DA6013BD1A6816494C
:101BA0000A40C5E7086802430A6014221A701A78CE
:101BB000002ACED01A78013AD2B2F7E7C8680243B9
:101BC000CA6014221A7019784A1ED2B21A700029FB
:101BD000F9D1C4E71A78013AD2B2C7E71A78013AC4
:101BE000D2B2CEE74C45FF1F1446FF1F3CF0004029
:101BF0004445FF1F00200040FFFFFEFF564B70B51D
:101C00001B68012B03D1554A936D0133936502F094
:101C100013F9534B534A1860534B544C1A60012329
:101C2000534A1360534A13602378002B06D00622D0
:101C30005149524802F040FA00232370504A514B58
:101C400010681B78C1B2002B0ED14F4CC0B2237864
:101C50005BB2002B4FDB237824785BB264B21B04A9
:101C600024021B191B1813600B1C50294ED950233A
:101C7000464A47491078DBB2FF2202284BD1086858
:101C8000444C454D267890432A78964254D9227880
:101C900024782E78023B5D10A31B6B435201D31AAC
:101CA00010335B111843086002F0F6F8031F012B94
:101CB00045D83A4B1B78002B06D0394B1B78002BAC
:101CC00002D0002002F0F0F9A122364B9200997860
:101CD000354B4A431B689B18832292009B181B7844
:101CE000033B012B03D8AF20400002F0BDF90122D5
:101CF0002E4BDA8270BD237824785BB264B2FF3356
:101D0000FF341B0424021B190138ABE7CAB2022AB4
:101D1000AED20223ACE70868254C264D26789043C6
:101D20002A78964208D9227824782D78023B5B10D5
:101D3000641B63435201B2E72378DBB2B2E70228A7
:101D4000D5D11D4B1B78013B022B03D91B4B1B78B4
:101D5000022BCCD16C20C8E79809FF1FFC0FFF1F96
:101D60005466FF1FFF3F0000141003405866FF1F1A
:101D70000C10034000100340D50BFF1F7211FF1F12
:101D8000B40003408C09FF1F680AFF1F490AFF1FA8
:101D900094000340460AFF1F470AFF1FF908FF1F70
:101DA0002209FF1F300DFF1F3409FF1FBC0BFF1F4F
:101DB000440AFF1F450AFF1F1C09FF1F2309FF1FBD
:101DC00010B502F019F80022014B1A8010BDC04670
:101DD0005066FF1F10B502F07FF8A121054A890067
:101DE0009478054A61431268044B5218528C1A8049
:101DF00010BDC046300DFF1F3409FF1F5066FF1F86
:101E000010B50D4B0D4A9978A1239B004B431268E6
:101E1000D218531DD97F0A4B1B88994209D2441C02
:101E200007D0C82805D0D2695B1A5A43054B5343E3
:101E3000C01802F0C9F910BD300DFF1F3409FF1F93
:101E40005066FF1F7102000070B5244D2B68002BF7
:101E500028D002F0A1F82B68D8402B680400002B92
:101E600027D001F051FF2B68D8401D4B1D4A9978AF
:101E7000A1239B004B431268D118D25C91239B0095
:101E8000002A20D0CA580132CA50174B17491B6884
:101E90000868834214D3D23B181A012A1AD0144B73
:101EA000186070BD02F078F8124B196801F06CFFF1
:101EB000D3E701F029FF0F4B196801F065FFD4E764
:101EC0000D495B18E8E7CA500C4B1B68DB68E41847
:101ED000201AE4E7F530FF30E1E7C0461C08FF1F99
:101EE000300DFF1F3409FF1F9C09FF1F5466FF1FA1
:101EF000A009FF1F1808FF1F2DFF3F005C66FF1F92
:101F000070B504000D00282916D10300A433C2883F
:101F10001B889B1A0B4A9BB293420DD906006A3666
:101F200005223100653001F037FF002804D131006F
:101F3000200002F059F970BD2900200001F08CFF4B
:101F4000F9E7C046FE7F0000F8B50400012002F06A
:101F50007BF801F0F1FF0300184A19491060886A04
:101F60008D6AA842FBD1174D174E28607568AC46A4
:101F7000164D2F680025BC4501D275687D1B144E97
:101F800000193560C862A4204C6A400320434862AF
:101F900010490978002905D00F490978022902D192
:101FA0000F3B1360F8BD012901D1083BF9E7032974
:101FB00001D1053BF5E7033BF3E7C046E408FF1F0B
:101FC00000F00040340AFF1F28100040180AFF1FCD
:101FD0001C0AFF1F1C09FF1F4A0AFF1F70B580243F
:101FE0001025E405A3682B43A36001F0BDFFA3689F
:101FF000AB43A36070BD0000F7B5160080221C0043
:102000001023D2050191916805000B4393600022D3
:102010005A4BD7301A6001F06FFF9D232A002F0022
:102020009B00EB58CA3201210092FC37002B01D0F3
:102030000021009A386801F01FFF2900009BCB3176
:102040001A784F4BD3351A604B780A781B0213432A
:102050008A7812041A43CB781B061343494A1BBAE9
:1020600013604B790A791B0213438A7912041A43CD
:10207000CB7931001B061343434A1BBA13606B78BC
:102080002A781B021343AA7812041A43EB781B0622
:1020900013433E4A1BBA1360019A330213433C4A6E
:1020A00013603C4B22001B1B9C4603293DDCB308FC
:1020B0009A0013005142B21A032A46D1354AE01859
:1020C000511A82784078120400020243E05C043323
:1020D00002430A600022FF2B4BDDF0222E4B12013F
:1020E0001A600F222D4B1A602D4A1368002BFCD06A
:1020F0000023224A27491360091B321D0B191B6854
:10210000043A180A23706070180C1B0EA070E3705C
:102110000434002AF2DC802210213B68D20501330E
:102120003B6093688B439360F7BD6346D5789818FE
:1021300093782D061B042B43157804392B435578CF
:1021400004322D022B430360AFE7022A0AD1114A61
:10215000E05C511AE2185278120202430A6004331A
:102160009BB2B7E7012AB5D10A4A521AE15C116065
:10217000F5E7084959180A600433ACE70000044049
:102180003C00044038000440340004403000044067
:102190000C0004400001044004000440100004400E
:1021A00014000440F7B5150080221C001023D2054E
:1021B0000091916807000B4393600023654AD73074
:1021C000136001F099FE9D233E009B00F9583B00EF
:1021D000CA363200FC33002900D07FE0586801F095
:1021E0004BFE390032785C4BCB311A604B780A7861
:1021F0001B0213438A78AC4612041A43CB78281D7D
:102200001B061343554A1BBA13604B790A791B020C
:1022100013438A7912041A43CB791B061343504A9D
:102220001BBA13604B7A0A7A1B0213438A7A120490
:102230001A43CB7A21001B0613434A4A1BBA136088
:10224000009A2B021343484A13602200474B1B1B82
:102250000093009BCE785B1801938B7836061B04A5
:1022600033430E78043833434E7804313602334317
:10227000019E33600328ECDC0321A808431C9B006B
:102280002940800003292BD13849E5185E18A97828
:102290006D78E35C09042D02294319433160030082
:1022A00008330021FF2B2DDD314B324919600F21FE
:1022B000314B1960012327490B60304B1968002905
:1022C000FCD006211B680B40042B20D0802200206C
:1022D000D20593680A318B439360FEBD01217DE7EF
:1022E000022908D121495D18E1184978E35C090207
:1022F00019432960D3E70129D3D11C495918E35C5C
:102300000B60CCE71948181801600433CAE70023B2
:1023100010490B606346002B0CDC3B00FC335A6811
:10232000102101325A608022D205936801208B432C
:102330009360D2E7009B9B181B68190A13705170B9
:10234000190C1B0ED37004235B4291709C44043221
:10235000E0E7C046000004403C0004403800044070
:1023600034000440300004400C00044000010440EC
:1023700004000440080F0000100004401400044052
:1023800070B5061E19D00222614B9B799343012B35
:1023900013D1604B1A78FF2A0FD15A78FF2A0CD13B
:1023A0009A78FF2A09D1DA78FF2A06D11A79FF2A0A
:1023B00003D15B79FF2B00D1A7E0574B0C201A7893
:1023C000012A08D00022554D1A702B781A00093ABC
:1023D000042A01D8212070BD5A1F012AFAD94C4C79
:1023E000A07B042800D990E0A279032A00D98CE0D0
:1023F000821E012A03D862881F2A00D885E0002E99
:1024000061D0012E00D080E0A288012AE2D0002B0A
:102410000AD10138032803D801F05AFC151D1915FB
:102420001F202E7001F040FD2B785A1E032A16D86B
:1024300000253B4B1D602823237501F02DFEA8428B
:102440002ED0A580C6E7022320202B70EAE70423C4
:1024500022202B70E6E7032321202B70E2E7073BC5
:10246000012BB7D82F4B1B68DB6A9B06B2D52E4BCE
:102470001A78002AAED1A27B911E012901D9002A27
:10248000A8D1022280211A702823284D890128789A
:10249000237501F089FC80212878890101F0BCFCBA
:1024A0000123A380224B1B78002B0AD0FA22802123
:1024B000204B92001B8809025A431C4B187801F0EC
:1024C00023FD002087E701F067FE2B78A680073BFD
:1024D000012B06D918482E7001F0CEFD1E2001F008
:1024E000E3FC114B114C1A78002A06D080210022FF
:1024F000207889011A7001F057FC01F00DFD802150
:102500002078090201F050FCDBE7122063E7C046A7
:10251000A60BFF1F6B09FF1F1A09FF1F1C09FF1FD6
:102520004809FF1F5C66FF1F2309FF1F1B09FF1FD0
:102530002109FF1F2C09FF1F0010004010B50029C2
:1025400001D001F039FC10BDF7B5604B01919978CD
:10255000A1239B004B435E4A060014681022E41836
:10256000D6235B00E0583623FF33E35C0027934318
:10257000222B41D1574B0F3A1A600760012501F019
:10258000BBFD019B1880E8235B00E35C002B01D0BE
:10259000B34258DD0023504FFB70AD33FF33E35897
:1025A0001A68002A03D09B88DB439B071DD0382381
:1025B000FF33E35C002B18D09B235B00E35C002B14
:1025C00013D1D133FF33E35CB3420EDAA4235B00B3
:1025D000E15AE018090A023101F03EFD2300012210
:1025E000FE33013E01351A87FA70E8235B00E35C95
:1025F000002B2AD0A8B2FEBD03683D00002BBED040
:1026000081880430090A023101F026FDD6235B00DF
:10261000E3581F60B2E72300B133BA00FF33985884
:10262000013781880430090A023101F015FDE823E1
:102630005B00E35CBB42EEDCE822F61AED180023F7
:102640005200A354A6E70027F1E7200001F00CFC9C
:1026500000281FD0002E1DDD73198826471901930D
:10266000B600200001F090FD5A308000201840682C
:10267000013581880430090A023101F0EDFC2000A7
:1026800001F022FDA3590133A351BD4202D0019BA9
:102690009D42E6D1114BE35C002BABD095239B0010
:1026A000E35C002BA6D00E4BE15A0029A2D00D4AC4
:1026B000A35C994202D90133A3549BE700231A215A
:1026C0002000A35401F028FD94E7C046300DFF1F01
:1026D0003409FF1F00140340E010FF1F5A020000DE
:1026E000720200005E020000F8B51D4B1D4F1A7803
:1026F000002A10D1BA7B002A02D101321A7003E0FD
:10270000032AFAD0022AF8D001F0C6FC00220120E8
:10271000154B1A70F8BD154B154D1C68154B9E785E
:1027200001232B702878C0B200F0CEFCBB7B002BBD
:102730000BD101F0F9FBA1239B007343E418832321
:102740009B00E41823782B70E4E7032B02D101F0FF
:102750005BFCF0E70020022BDCD101F065FDEAE72D
:102760001C09FF1FA60BFF1F2309FF1F3409FF1FB2
:10277000490AFF1F300DFF1FF0B587B00EAD2F784F
:102780000FAD2D780593AC46634614000E4D0CAA90
:1027900012782E7803930D9B009201932200059BE3
:1027A000029701F001FC2E70012C01D0042C08D1FD
:1027B000802206498B889343054A1278D20113433D
:1027C0008B8007B0F0BDC0461C09FF1F6C11FF1FB6
:1027D0007809FF1F0B001B3B70B504003020E02B75
:1027E0000DD81300E025493BFF3B9BB2ED00AB4207
:1027F00005D8034B200019825A8201F005FB70BDF9
:102800008410FF1F10B501F017FB054B00205B681B
:10281000052B04D9034A5268D20200D4980810BD8F
:1028200000100040FCE100E070B501F0B5FC0D4B7C
:102830001B68FC33DC691D6AFFF7E4FF64198442FE
:1028400004D2094B01241B68002B07D0042200246A
:10285000064B1A70064A93690133936101F05CFBE1
:10286000200070BD5C66FF1F9809FF1F2309FF1F32
:10287000FC0FFF1F70B50C4D2B68FC335C6A01F038
:102880008BFCFFF7BFFF2B680025FC339B6AE31826
:10289000834204D2054B1B68AB4200D1051B01F0FB
:1028A0003BFB280070BDC0465C66FF1F9809FF1FF8
:1028B000D722044B92009B5810B5002B00D09847AC
:1028C00010BDC0460000FF1FF0B587B001F08AF9C7
:1028D000FFF7EEFFC54BC64C04931B78022B45D186
:1028E000C44B1B68186A01F0AFFBC34BC34A1A60A4
:1028F000C34BC44A1A60A022C34B52001A60049B07
:10290000187801F069FBC149C14801F015FCC149C3
:10291000C14801F011FC1022C04BFF201A60802238
:1029200052031A60802292031A60802212041A60F5
:1029300001F0BAFB012001F00FFCFA20400001F089
:102940003BFC582001F090FBB54801F035FB01201D
:1029500001F0FAFB072001F0BFFBE26DB14B1A401A
:1029600084235B001343E36507B0F0BD01F034FA44
:10297000AD4E0290322001F067FB33681B0628D46D
:102980003C2001F061FB0F2001F05EFB974B1B78B0
:10299000012B00D113E1802533682B4200D0A1E048
:1029A000636C03202B43636401F04EFB01F014FAC7
:1029B000029B0299C31A5A1E814200D81A009B4BEF
:1029C0001A608C4B19681E235343994A9B18CB619C
:1029D0008BE701F001FA8023E26BDB0213430390E3
:1029E000E363E26D8F4B03201A4028231343E36512
:1029F00001F02AFB0320A56E01F026FBA36E032045
:102A0000DB03DB0B019301F01FFBA76EED03FF035C
:102A1000ED0BFF0B874AAB18C22B2ED8019B9B18DE
:102A2000C22B2AD8BB18C22B27D8019B2A009D4253
:102A300000D21A00019B9D4200D91D003B00974225
:102A400000D21300BD4200D93D005B1B122B14D8ED
:102A50000C2233681420934333603368764A134062
:102A6000336001F0F1FA0821A36EE26DDB038A43C3
:102A7000E265724ADB0B136085E7032001F0E4FA9C
:102A8000A36EDB03DB0B059301F0A6F9039B03990F
:102A9000C21A531E814200D81300694A93421BD9BF
:102AA000FF23356864492D0A1D4032686B1C1B06E4
:102AB0000A401B0C134333600C23326800209A43F6
:102AC000083B1343336001F087FB5E485E4BA84030
:102AD000984205DCFEF736FF019D0197059F99E7B7
:102AE0005A48F7E700235A4E33608023226CDB02FA
:102AF00013432364636C03202B43636401F0A4FA43
:102B00003368013333608023626C5B021343636478
:102B100005230193E26D434B03201A404D4B1343B1
:102B2000E36501F091FA0821A26EE36D434F8B43F8
:102B3000E3653B6802394B43D203D20B9A420CD86F
:102B40009B1A3B2B0BD8E36D43490B40E365636C49
:102B50000B406364414B1A6028E7D31AF1E7019BED
:102B6000013BDBB20193002BD4D1E36D3A4A134011
:102B7000E365636C134063643368042B07D9BFF3C8
:102B80004F8F374B374ADA60BFF34F8FFEE7636CE6
:102B90000320AB43636401F057FAE26D214B03203D
:102BA0001A4028231343E36501F04EFA0822A36E6E
:102BB000DB03DB0B3B60E36D9343E3659AE707229E
:102BC000E36B1340012B02D1002001F005FA264DE2
:102BD000264AAB6802201340AB6001F035FA80232F
:102BE000AA685B001343AB60E0E6C0464A0AFF1FD9
:102BF00000F000405C66FF1F000003400180063DBE
:102C0000BC00034034080000A4000340710200002F
:102C100014100040FFFF3F002810004000E100E0DA
:102C20003075000000FEFEFFC4F000404466FF1F48
:102C30007206000091FCFFFFFF00FFFF4C66FF1FC4
:102C4000E30C0000E88000005F361E0060361E00C6
:102C5000B044FF1F28000100FFFFFEFF4866FF1F72
:102C600000ED00E00400FA053CF00040FFFEFFFF2D
:102C7000694E336888331B6883F3088801F0C4FA0F
:102C800000F018FC654B664A1B68934207D0002091
:102C900001F0A2FA0221634A13688B431360FFF725
:102CA00013FE614B614C1878C0B201F04DF800235F
:102CB000A3600233A3605E4B0120236001F0C4F9DE
:102CC0000323A36001F088F8040001F0B5F80500C3
:102CD00001F082F8574B186001F056F9564B19680D
:102CE000621A531EA14200D213008022D2039342E3
:102CF00001D39B029B0A3268D16AC90700D478E0ED
:102D00004E491C0C09689BB24C4359432402090AE2
:102D1000641803274A49FC3293680A6849489B1A99
:102D2000494A4A4E12684A499B18414A34609A18E7
:102D30003B400193036892089C46019B0A606344F0
:102D40000360042B03D901323B400A6003600B6827
:102D50004049E418200001F017F83F4F3D493B6817
:102D6000C3183B602000019301F066FA3B4C2068D9
:102D7000081838492060884205D9019B01333B601F
:102D800001F05AFA216001F0E7F8354B1B78002B6F
:102D90000ED001F051F83168324B4A1B1B681218F3
:102DA0009A4233D2591A4919091A2F4801F0C4F925
:102DB0002E4C237A002B0FD001F03EF83168E368E7
:102DC0004A1B1218934224D9591A4919091A28483A
:102DD00001F0B2F900232372264B83F3088800F038
:102DE0009BFF022001F060F8002001F0F5F901F0EE
:102DF0002BF8DC0199000234641A5900641A092185
:102E00004B438033CB40A408E41882E7FA218900C1
:102E1000CBE71949DBE7C0465C66FF1F0C0AFF1FC2
:102E2000B641210310000040490AFF1F1410004062
:102E3000C4090000100AFF1F340AFF1F380AFF1FD1
:102E4000200AFF1F280AFF1F1C0AFF1F4066FF1FE2
:102E5000240AFF1F710200006008FF1F2C0AFF1FD9
:102E60001C09FF1FE408FF1F00100040740BFF1F28
:102E70003C10004000000020DC050000A022054BB3
:102E800092009B5810B5002B01D0984710BD01F05F
:102E9000FBF8FBE70000FF1FA122054B92009B58A7
:102EA00010B5002B01D0984710BD01F0EDF8FBE7FD
:102EB0000000FF1FA222054B92009B5810B5002B6B
:102EC00001D0984710BD01F0DFF8FBE70000FF1FBD
:102ED000A322054B92009B5810B5002B01D09847B8
:102EE00010BD01F0D1F8FBE70000FF1FA422054B45
:102EF00092009B5810B5002B01D0984710BD01F0EF
:102F0000C3F8FBE70000FF1F70B500F095FF514BC1
:102F10001860042000F0C8FF00F02EFF0400C30773
:102F200002D400F019FF70BD00224B4B1A604B4BCE
:102F30001878013804282CD800F0CAFE03231B1F80
:102F40002700200000F070FF0128ECD0444C2378CB
:102F5000042B71D100F008FF002806D000F034FFE8
:102F6000582001F081F802232370032000F09CFF19
:102F7000D9E7200001F050F9E6E7200001F024F83D
:102F8000E2E7200001F010F9DEE7200001F0ECF8A4
:102F9000DAE700F081FF0500012808D1314B1B78EA
:102FA000053B012B03D82000FFF768FFCEE72C4B31
:102FB0001B78022B01D0052B20D1022D28D12A4BC2
:102FC0009B7BAB431CD12000FFF766FF254B187895
:102FD0000128BBD16405B9D4234925224B7B034288
:102FE00005D1233A13405A42534126331A000B7D30
:102FF0009342ABD9322000F0A7FFA7E7022D07D1FB
:10300000184B1B78052B11D12000FFF753FFDDE78C
:10301000012D0BD1012B03D12000FFF759FF95E7BC
:10302000062B03D12000FFF761FF8FE7200001F09E
:103030002BF8022D8AD1C9E7032B04D10B4B987CC6
:1030400000F052FF91E7072B8FD1094B987B00F0DE
:103050006BFE8AE79C09FF1F9809FF1F9009FF1F5D
:103060002309FF1F1C09FF1FA60BFF1FBC0BFF1F1F
:10307000D40BFF1FFA210A4B0A4A49001A640A4A74
:103080005A500A4A04395A50094A08319A64094A7E
:103090005A50094A5C315A50084ADA667047C046AD
:1030A0000000FF1F7927FF1F7528FF1F2928FF1F1A
:1030B0008123FF1FE926FF1F011EFF1FD51DFF1FD4
:1030C00010B500F0EDFD10BD8023F7B59C46264BF2
:1030D000264F01932649274A274D284C284B022882
:1030E0001AD1604638600868264E30408026360384
:1030F0003043086001990978002909D11660224AF5
:103100002A60224A2260E02219689143A03A1BE01B
:103110008021C9021160F2E766463E600F68194ED1
:103120003E408027FF023E430E6001990978002946
:103130000DD1176001280ED1154A2A60154A226068
:10314000E02219689143C03A0A431A60F7BD802112
:1031500089021160EEE7E0210F4A02432A600F4A1C
:1031600022601A688A43F0E74B0AFF1FE000034021
:10317000D80003409000034000000340500003408B
:1031800040000340FFFFE3FF0280063D8045082228
:103190000180063D8066082200800698805508223E
:1031A000F8B51E4B80261A680020140034403242C5
:1031B00032D11A681A4F32431A6001223B68063036
:1031C00093433B6000F040FF0122164D2B681E43E5
:1031D0002E603B680A2613433B608027BF00124BDA
:1031E0001B683B4211D1013EF6B2FF2E09D17E226F
:1031F0000E4B1C682B68E40B1440934323432B6055
:1032000005E0082000F020FFE9E7002EEFD1802242
:103210002B68600893432B60F8BDC046C4F00040A3
:103220005CF0004018F0004068F0004060F00040A2
:1032300010B500F069FF01215820034A00F03CFE60
:10324000FFF7AEFF10BDC046600AFF1F10B5782221
:103250000021034800F0D0FE00F04EFD002010BD1C
:103260006469FF1F70B5040000F096FF00230C2076
:103270000B4A010059438D18515C00290DD0A14221
:1032800008D1012300246B7000F02EFF00F044FEF3
:10329000200070BD01330A2BEBD11224F6E7C046A3
:1032A0006469FF1F70B5040000F076FF0023190069
:1032B0001D000D4A1078002806D0A0420CD1557090
:1032C00001310C320A29F5D1002B0AD100F014FD8E
:1032D00000F022FE002070BD5078461EB0411B1841
:1032E000EEE700F001FFF3E76469FF1FF7B50400A4
:1032F0000C20002384460E4D019267465F43E85D33
:103300007E19A04212D000280BD10A4B9C4662467F
:103310001B7808331370019B70707C557160B3602B
:10332000FEBD01330A2BE8D10320F9E70720F7E7B8
:103330006469FF1F6069FF1F8020F8B5484BC00516
:103340001B68C1248360474BFF251A680123134380
:103350004361454BA4001A68444B40211A60444B1A
:103360001A68444B1A60444B1A59AA431A51C52291
:1033700092009E58AE433143802699509F583F4952
:10338000F6010F403E439E509E5880273602360A73
:103390003043985080201A5900020A4002431A51C3
:1033A00004341A59364E3F04324080263A431A51AB
:1033B0001A5936061202120A32431A5108341A599F
:1033C00080260A4002431A51C32292009F58B446F5
:1033D000AF4337439F509F58294E0F4007439F509C
:1033E0009F58374080263604374380269F509F5889
:1033F00036063F023F0A37439F50C0221F59AF4352
:103400003A431A511A591202120A1643C6221E5181
:1034100092009C58AC4365462C439C509C58002518
:103420000C4020439850C72080001A58154C11407A
:10343000C02212020A431A50134B1B78DB08AB421E
:1034400001DC0020F8BD2378002B06D0A368002BF8
:1034500000D0984701350C34EEE71220F2E7C04661
:103460004845FF1F4445FF1FB0F000405C69FF1F47
:10347000B4F000405869FF1F00E100E0FF00FFFFCB
:10348000FFFF00FF6469FF1F6069FF1F030010B5A5
:103490001F2809D8072200201340072404490A786E
:1034A000A24313430B7010BD00230620F5E7C0466E
:1034B0006069FF1F034A0449136800200B40136032
:1034C0007047C0461CF00040FFFFC1FF054B064996
:1034D0001B780A6805485B0702401B0B134300205A
:1034E0000B6070476069FF1F1CF00040FFFFC1FFC9
:1034F00070B50C25FFF7EAFF0A4B1C780A4BE4086D
:103500006543ED18002C01D1200070BD2B78002BF5
:1035100006D06B68002B00D09847013C0C3DF1E7CA
:103520001220F2E76069FF1F5869FF1F07B50422E8
:10353000074801A900F034F9019B013305D180232C
:10354000044ADB0411680B43136000200EBDC04623
:103550001C18001114F00040F0B505002026184B8F
:1035600087B00493049B002B03D11124200007B0E3
:10357000F0BD002102220B0001910091052000F016
:10358000DBFB02230F490A681A42FCD10596059C11
:10359000631E0593002CFAD10B4A1368002BFCDA4A
:1035A0000F276F440121380000F03EFD3B782B428D
:1035B000DCD0052000F048FD049B013B0493D1E7DB
:1035C000FFFFFF0790C8004000C8004007B500F0AB
:1035D000E3FD80220821D205936A0191002B01D1DD
:1035E0000739916202210C4A11600199481E01902D
:1035F0000029FAD103311160053101910199481E6A
:1036000001900029FAD11160002B02D18022D2054D
:10361000936200F081FC07BD00C00040F0B52D4C66
:1036200089B02378002B4FD1FEF76CF902232A4F83
:1036300003903A681A42FCD120230693069B5A1E37
:103640000692002BFAD1254E3368002BFCDA0120BC
:10365000FFF782FF011E02D0112009B0F0BD030068
:1036600003220190009005AD9F2000F065FB03212F
:10367000280000F0D9FC02233A681A42FCD120232A
:103680000793079B5A1E0792002BFAD13368002B31
:10369000FCDA0120FFF760FF0028DDD10398FEF778
:1036A00045F9AA786B7811041B020B4329780B4368
:1036B00063601300113B0A49052B07D8012393408F
:1036C000A3600B60012323700020C6E780231B0347
:1036D000F6E7C0463045FF1F90C8004000C80040D4
:1036E0009808FF1F1E4B30B55A6818781D4B85B0DF
:1036F000D31859424B4101210093002300F0C4FB31
:10370000194B1A4A02259A6300221A6510325A652B
:103710008022C4219D65164B1648D202DA678900C3
:103720004258154B80241A4080231B0413434350F6
:10373000642341200393E40500F078F9402000F071
:1037400075F96562039D6B1E0393002DFAD1032367
:103750006362FFF73BFFA562FFF760FF05B030BD76
:103760003C45FF1F95FFFEF700C80040050001FF24
:1037700004E100E000E100E0FFFF00FF10B5064BB0
:1037800018705960FFF7AEFF00211320034AFFF7BE
:10379000ADFD002010BDC0463C45FF1FE536FF1FB4
:1037A000F0B5040085B003920291FEF7ABF88822D1
:1037B00063035B0B52051A438023DB059D6A80235C
:1037C000274F0092BA68002601901B039A420CD939
:1037D000F82326001B041E401C4206D08022214BE9
:1037E00052025E6219680A431A60002D0BD100F084
:1037F000D3FC02221C4B1A608023DB055A62013A7B
:103800009A6200F089FB0023039A934220D1002D95
:103810000AD100F0C1FC144B03221D608023DB059C
:103820005A629D6200F078FB8023BA681B039A42BB
:1038300008D9002E06D000220A4B0C495A621A6899
:103840000A401A600198FEF771F8002005B0F0BD3B
:10385000009A0299D2181278CA540133D4E7C046AC
:103860003045FF1F00C8004000C00040FFFFFEFFC2
:10387000F0B587B0029103920400FEF743F801907F
:1038800000F08AFC802302250122234EDB053560EF
:103890005D629A6200F040FB204F3B682B42FCD1F6
:1038A00020230493049B5A1E0492002BFAD11C4D32
:1038B0002B68002BFCDA0120FFF74EFE002802D017
:1038C000112007B0F0BD2000039A029900F054FBCC
:1038D000022304003A681A42FCD120230593059B79
:1038E0005A1E0592002BFAD12B68002BFCDA01201E
:1038F000FFF732FE051EE3D100F04EFC80230322C9
:10390000DB0535605A629D6200F006FB0198FEF708
:103910000DF8E0B2D5E7C04600C0004090C80040B6
:1039200000C80040F0B5802687B00400FDF7EAFF2C
:10393000F605B36A02250393029000F02DFC0123E3
:10394000244F3D607562B36200F0E6FA224E3368A0
:103950002B42FCD120230493049B5A1E0492002B7B
:10396000FAD11E4D2B68002BFCDA0120FFF7F4FD85
:10397000002802D0112007B0F0BD200000F0A4FA0A
:103980000223019032681A42FCD120230593059B43
:103990005A1E0592002BFAD12B68002BFCDA03206B
:1039A000FFF7DAFD041EE5D100F0F6FB80230322C9
:1039B000DB053C605A629C6200F0AEFA039B002B70
:1039C00001D1FFF703FE0298FDF7B0FF6B461879AF
:1039D000D1E7C04600C0004090C8004000C8004089
:1039E00007B5000201910422000A01A9FFF740FF78
:1039F0000EBD000073B5050005240B4AA3005B4211
:103A00009B1819686B46DE1D300000F0EDFA0228A5
:103A100004D133782B55013CEFD276BD052CFCD078
:103A20000128FAD10230F8E7140900111F2807D83D
:103A3000012380228340D20591680B439360704735
:103A40003F2808D80123802220388340D2055169BD
:103A50000B435361F3E75F28F1D8012380224038FC
:103A60008340D205116A0B431362E8E71F2807D889
:103A7000012280218240C9058B6893438B60704787
:103A80003F2808D80122802120388240C9054B698F
:103A900093434B61F3E75F28F1D80122802140383E
:103AA0008240C9050B6A93430B62E8E71F2810D8D0
:103AB00080230200DB05153A1968012A06D8202266
:103AC0009143196019680A431A60704701228240C5
:103AD000F6E73F2811D880230200DB05353AD96884
:103AE000032A06D810229143D960D9680A43DA60C4
:103AF000EBE7012220388240F5E75F28E5D8422332
:103B00008022181A413B8340D205516A9943516281
:103B1000516A0B435362D8E710B50400012813D152
:103B2000A022184992050B685B015B0913430B60E7
:103B3000154B164A19681140154A0A431A6040226B
:103B400019680A431A6010BD0028FCD101000A2040
:103B500000F062FA21000B2000F05EFAC0220A4B4E
:103B6000920019680A4340211A601A688A431A6051
:103B7000B022044912060B685B015B0913430B601A
:103B8000E1E7C04614F000401CF000407F00FEFF5B
:103B900080FD010072B6074A1368013313600422E6
:103BA000054B1A600023054A13608022D20553603A
:103BB000FEE7C0467808FF1FC0F00040C4F0004098
:103BC000044B054A1A60054B1A600022044B1A6028
:103BD0007047C046140AFF1F841E0000380AFF1FEA
:103BE000C4F000400023034A1360034A1360034AF1
:103BF0001360704754F0004040F1004044F1004031
:103C0000002310B5184C8AB0009301932378012B40
:103C100027D06946012000F0EFFA002817D1009B59
:103C200012490293019B06AA0393114B02A81B6839
:103C30000493104B1B68059300F096F910220E496F
:103C400006A800F0A9F8002804D1FF232370002063
:103C50000AB010BD0123094A074902A8237000F0E9
:103C600083F90120F4E7C0466066FF1F10290011A8
:103C7000082900110C290011202900116466FF1F7A
:103C800013B501246946012000F0B6FA034B0094F5
:103C90000193FFF7B5FF200016BDC046BB0B000027
:103CA00010B5FFF79FFFFFF7EBFF002802D0024B94
:103CB000984710BDFEE7C046E1A2000002B471467D
:103CC00049084900095649008E4402BC7047C04665
:103CD00002B4714649084900095C49008E4402BC9F
:103CE0007047C04603B47146490840004900095A6C
:103CF00049008E4403BC704701B40248844601BCAD
:103D0000604700BFADAE000001B40248844601BC6C
:103D1000604700BF6D0B010001B40248844601BC3E
:103D2000604700BF7997000001B40248844601BC97
:103D3000604700BFC1F7000001B40248844601BCDF
:103D4000604700BF496D010001B40248844601BCD0
:103D5000604700BF8914010001B40248844601BCD9
:103D6000604700BFDD0A010001B40248844601BC7F
:103D7000604700BF01D7000001B40248844601BC7F
:103D8000604700BFBD0B010001B40248844601BC7E
:103D9000604700BF090E000001B40248844601BC20
:103DA000604700BFCD4C010001B40248844601BC0D
:103DB000604700BFB352010001B40248844601BC11
:103DC000604700BFE9D4000001B40248844601BC4A
:103DD000604700BF6DF6000001B40248844601BC94
:103DE000604700BF156B010001B40248844601BC66
:103DF000604700BFF9A6000001B40248844601BC38
:103E0000604700BF8D82000001B40248844601BCB7
:103E1000604700BF116E000001B40248844601BC37
:103E2000604700BF0D52010001B40248844601BC46
:103E3000604700BF0134010001B40248844601BC60
:103E4000604700BFC95C010001B40248844601BC60
:103E5000604700BF8552010001B40248844601BC9E
:103E6000604700BF51B8000001B40248844601BC5D
:103E7000604700BF71B0000001B40248844601BC35
:103E8000604700BF2144000001B40248844601BCE1
:103E9000604700BFC56D010001B40248844601BC03
:103EA000604700BFDD0C010001B40248844601BC3C
:103EB000604700BF1907010001B40248844601BCF5
:103EC000604700BF0167010001B40248844601BC9D
:103ED000604700BFA96F010001B40248844601BCDD
:103EE000604700BFF9ED000001B40248844601BC00
:103EF000604700BF4DF9000001B40248844601BC90
:103F0000604700BF8944000001B40248844601BCF8
:103F1000604700BF8B52010001B40248844601BCD7
:103F2000604700BF9DA9000001B40248844601BC5F
:103F3000604700BFE9F6000001B40248844601BCB6
:103F4000604700BFBD5C010001B40248844601BC6B
:103F5000604700BF6137010001B40248844601BCDC
:103F6000604700BFD544010001B40248844601BC4B
:103F7000604700BFDD3F000001B40248844601BC39
:103F8000604700BF9573010001B40248844601BC3C
:103F9000604700BFC166010001B40248844601BC0D
:103FA000604700BFE90B010001B40248844601BC30
:103FB000604700BF9D6A000001B40248844601BC0E
:103FC000604700BF8D11010001B40248844601BC66
:103FD000604700BF0534010001B40248844601BCBB
:103FE000604700BFEDA5000001B40248844601BC53
:103FF000604700BF9938001101B40248844601BCF3
:10400000604700BFB70E000001B40248844601BCFF
:10401000604700BF75F8000001B40248844601BC47
:10402000604700BF89A2001101B40248844601BC68
:10403000604700BF3D71010001B40248844601BCE5
:10404000604700BFA1AF000001B40248844601BC34
:10405000604700BF0189000001B40248844601BCEA
:10406000604700BFC115010001B40248844601BC8D
:10407000604700BF7912010001B40248844601BCC8
:10408000604700BFC1A5000001B40248844601BCDE
:10409000604700BFE917010001B40248844601BC33
:1040A000604700BFA9D8000001B40248844601BCA3
:1040B000604700BFED6B010001B40248844601BCBB
:1040C000604700BFE94C010001B40248844601BCCE
:1040D000604700BF5976010001B40248844601BC24
:1040E000604700BFF90D010001B40248844601BCDD
:1040F000604700BF21A9000001B40248844601BC0A
:10410000604700BFCD0C010001B40248844601BCE9
:10411000604700BFED68010001B40248844601BC5D
:10412000604700BF53B9000001B40248844601BC97
:10413000604700BFE927000001B40248844601BC83
:10414000604700BF2D6C010001B40248844601BCE9
:10415000604700BFE512010001B40248844601BC7B
:10416000604700BF6911010001B40248844601BCE8
:10417000604700BFF935010001B40248844601BC24
:10418000604700BF51B6001101B40248844601BC2B
:10419000604700BFD9B0000001B40248844601BCAA
:1041A000604700BF75A9000001B40248844601BC05
:1041B000604700BFF535010001B40248844601BCE8
:1041C000604700BF8512010001B40248844601BC6B
:1041D000604700BF8937010001B40248844601BC32
:1041E000604700BF016C010001B40248844601BC75
:1041F000604700BF85C1000001B40248844601BC8D
:10420000604700BFE1AC000001B40248844601BC35
:10421000604700BFC9A9000001B40248844601BC40
:10422000604700BF0934010001B40248844601BC64
:10423000604700BF19FA000001B40248844601BC7F
:08424000604700BF090E0000F9
:1042480002000000AABF0011010000005CBD0011BF
:1042580002000000A6BF0011010000008842FF1FF5
:104268000200000064BD001101000000A063FF1FF0
:1042780002000000A4BF0011030000001463FF1F28
:104288001200000002000000AABF00110100000097
:10429800A4BD001102000000A6BF0011010000002B
:1042A800A1BD001102000000AEBD00110300000016
:1042B8004F63FF1F02000000A4BF001103000000AD
:1042C8006463FF1F02000000A6BF00110100000088
:1042D800A0BD001102000000ACBD001103000000E9
:1042E8002563FF1F02000000A4BF001103000000A7
:1042F8004663FF1F02000000AABF00110100000072
:10430800E4BD001102000000A6BF0011010000007A
:10431800D143FF1F02000000F6BD0011010000009C
:10432800DFBD001102000000A6BF0011010000005F
:10433800D043FF1F02000000F4BD0011010000007F
:104348006C63FF1F02000000A6BF001101000000FF
:10435800CF43FF1F02000000F2BD00110100000062
:10436800CFBD001102000000A6BF0011010000002F
:10437800CE43FF1F02000000F0BD00110100000045
:10438800CABD001102000000A6BF00110100000014
:10439800CD43FF1F02000000EEBD00110100000028
:1043A800C5BD001102000000A6BF001101000000F9
:1043B800CC43FF1F02000000ECBD0011010000000B
:1043C800C0BD00110202020202020000000000004B
:1043D8000D0C00002D4C0011F34B001138BE0011DC
:1043E800900118001800FFFF0701020304050602E8
:1043F80001060000000000000000000000000000AE
:1044080000000000000000000000000000000300A1
:1044180002000000AABF001101000000B8BE001190
:1044280002000000A6BF0011010000008844FF1F21
:1044380002000000C2BE0011010000009A63FF1FC5
:1044480002000000A4BF0011030000000866FF1F5F
:1044580002000000A6BF0011010000008844FF1FF1
:1044680002000000C0BE0011010000009C63FF1F95
:1044780002000000A4BF0011030000000066FF1F37
:10448800126C6C6C0000000000580040151600000B
:104498000001000000000111FFFF000050485936DC
:1044A80000000000000000000100000049BE0011EB
:1044B8000B000500F7000000B400002800280028C1
:1044C8003075A000A000A000A00000080008E001CE
:1044D800F000100010001000100010001000500034
:1044E8005000500010001000D0070000000000002D
:1044F8000F0001000500307507001000010081FF62
:1045080000000000FF0000007174001179720011B2
:1045180009700011FFFF0100FF0000008D9E0011CF
:10452800099C0011219B0011000000000000000000
:1045380000000800040000003B0001085902E001E7
:1045480088212800FF00000002000000AABF001117
:104558000100000070C0001102000000A6BF001199
:1045680001000000CD45FF1F02000000A2BF00119E
:10457800010000001C6AFF1F02000000A6BF001116
:1045880001000000CC45FF1F02000000A0BF001181
:1045980001000000CA45FF1F02000000A6BF00116D
:1045A80001000000C845FF1F020000009EBF001167
:1045B80001000000C045FF1F18001800000090010E
:1045C800020000030202000002000000AABF00115E
:1045D8000100000084C0001102000000A6BF001105
:1045E800010000001046FF1F020000009CBF0011E0
:1045F800000000000000000002000000A4BF00113D
:0A460800030000003C6AFF1F20FFC2
:040000051FFF184180
:00000001FF
